Archive member included because of file (symbol)

c:/program files/microchip/mplab c30/bin/bin/../../lib\libpic30-coff.a(crt1.o)
                              (_resetALT)
c:/program files/microchip/mplab c30/bin/bin/../../lib\libpic30-coff.a(crt0.o)
                              (_resetPRI)
c:/program files/microchip/mplab c30/bin/bin/../../lib\libm-coff.a(floatsisf.o)
                              Objects - Image Decoders Demo\Application.o (__floatsisf)
c:/program files/microchip/mplab c30/bin/bin/../../lib\libm-coff.a(mulsf3.o)
                              Objects - Image Decoders Demo\Application.o (__mulsf3)
c:/program files/microchip/mplab c30/bin/bin/../../lib\libm-coff.a(addsf3.o)
                              Objects - Image Decoders Demo\Application.o (__subsf3)
c:/program files/microchip/mplab c30/bin/bin/../../lib\libm-coff.a(fixsfsi.o)
                              Objects - Image Decoders Demo\Application.o (__fixsfsi)
c:/program files/microchip/mplab c30/bin/bin/../../lib\libm-coff.a(modsi3.o)
                              Objects - Image Decoders Demo\BmpDecoder.o (__modsi3)
c:/program files/microchip/mplab c30/bin/bin/../../lib\libm-coff.a(divsi3.o)
                              Objects - Image Decoders Demo\BmpDecoder.o (__divsi3)
c:/program files/microchip/mplab c30/bin/bin/../../lib\libm-coff.a(udivsi3.o)
                              Objects - Image Decoders Demo\FSIO.o (__udivsi3)
c:/program files/microchip/mplab c30/bin/bin/../../lib\libm-coff.a(umodsi3.o)
                              Objects - Image Decoders Demo\FSIO.o (__umodsi3)
c:/program files/microchip/mplab c30/bin/bin/../../lib\libm-coff.a(fpack.o)
                              c:/program files/microchip/mplab c30/bin/bin/../../lib\libm-coff.a(floatsisf.o) (_fpack)
c:/program files/microchip/mplab c30/bin/bin/../../lib\libm-coff.a(funpack2.o)
                              c:/program files/microchip/mplab c30/bin/bin/../../lib\libm-coff.a(mulsf3.o) (_funpack2)
c:/program files/microchip/mplab c30/bin/bin/../../lib\libm-coff.a(futil.o)
                              c:/program files/microchip/mplab c30/bin/bin/../../lib\libm-coff.a(mulsf3.o) (_fPropagateNaN)
c:/program files/microchip/mplab c30/bin/bin/../../lib\libm-coff.a(funpack.o)
                              c:/program files/microchip/mplab c30/bin/bin/../../lib\libm-coff.a(fixsfsi.o) (_funpack)
c:/program files/microchip/mplab c30/bin/bin/../../lib\libc-coff.a(rand.o)
                              Objects - Image Decoders Demo\Application.o (rand)
c:/program files/microchip/mplab c30/bin/bin/../../lib\libc-coff.a(srand.o)
                              Objects - Image Decoders Demo\Application.o (srand)
c:/program files/microchip/mplab c30/bin/bin/../../lib\libc-coff.a(memset.o)
                              Objects - Image Decoders Demo\FSIO.o (memset)
c:/program files/microchip/mplab c30/bin/bin/../../lib\libc-coff.a(strncpy.o)
                              Objects - Image Decoders Demo\FSIO.o (strncpy)
c:/program files/microchip/mplab c30/bin/bin/../../lib\libc-coff.a(toupper.os)
                              Objects - Image Decoders Demo\FSIO.o (toupper)
c:/program files/microchip/mplab c30/bin/bin/../../lib\libc-coff.a(tolower.os)
                              Objects - Image Decoders Demo\FSIO.o (tolower)
c:/program files/microchip/mplab c30/bin/bin/../../lib\libc-coff.a(strlen.o)
                              Objects - Image Decoders Demo\FSIO.o (strlen)
c:/program files/microchip/mplab c30/bin/bin/../../lib\libc-coff.a(strcpy.o)
                              Objects - Image Decoders Demo\FSIO.o (strcpy)
c:/program files/microchip/mplab c30/bin/bin/../../lib\libc-coff.a(strchr.o)
                              Objects - Image Decoders Demo\FSIO.o (strchr)
c:/program files/microchip/mplab c30/bin/bin/../../lib\libm-coff.a(mulsi3.o)
                              c:/program files/microchip/mplab c30/bin/bin/../../lib\libc-coff.a(rand.o) (__mulsi3)


Program Memory Usage

section                    address   length (PC units)   length (bytes) (dec)
-------                    -------   -----------------   --------------------
.reset                           0                 0x4             0x6  (6)
.ivt                           0x4                0xfc           0x17a  (378)
.aivt                        0x104                0xfc           0x17a  (378)
.text                        0x200               0x4a8           0x6fc  (1788)
.const                       0x6a8              0x23b2          0x358b  (13707)
.text                       0x2a5a              0x7f46          0xbee9  (48873)
.dinit                      0xa9a0                0x8a            0xcf  (207)
.isr                        0xaa2a                 0x2             0x3  (3)
__CONFIG2                  0x2abfc                 0x2             0x3  (3)
__CONFIG1                  0x2abfe                 0x2             0x3  (3)

                     Total program memory used (bytes):         0xff42  (65346) 24%


Data Memory Usage

section                    address      alignment gaps    total length  (dec)
-------                    -------      --------------    -------------------
_018e47e04a88ec30            0x800                   0           0x200  (512)
_018e46904a88ec30            0xa00                   0           0x200  (512)
.nbss                        0xc00                   0           0x1d6  (470)
.ndata                       0xdd6                   0            0x2a  (42)
.nbss                        0xe00                   0            0x24  (36)
.ndata                       0xe24                   0            0x12  (18)
.nbss                        0xe36                   0             0x6  (6)
.ndata                       0xe3c                   0             0x4  (4)
.bss                         0xe40                   0            0x88  (136)
.data                        0xec8                   0             0xa  (10)

                        Total data memory used (bytes):          0x6d2  (1746) 10%


Dynamic Memory Usage

region                     address                      maximum length  (dec)
------                     -------                      ---------------------
heap                         0xed2                               0xbb8  (3000)
stack                       0x1a8a                              0x2d76  (11638)

                        Maximum dynamic memory (bytes):         0x392e  (14638)


External Symbols in Data Memory (by address):

                    0x0800                  _gFATBuffer
                    0x0a00                  _gDataBuffer
                    0x0c00                  _defaultArray
                    0x0c0a                  _defaultString
                    0x0c18                  _gDiskData
                    0x0c36                  _cwd
                    0x0c6c                  _gFileTemp
                    0x0ca2                  _tempCWDobj
                    0x0cd8                  _dirCleared
                    0x0cda                  _TempClusterCalc
                    0x0cde                  _FSerrno
                    0x0ce0                  _FatRootDirClusterValue
                    0x0ce4                  _gTimeWrtDate
                    0x0ce6                  _gTimeWrtTime
                    0x0ce8                  _gTimeAccDate
                    0x0cea                  _gTimeCrtDate
                    0x0cec                  _gTimeCrtTime
                    0x0cee                  _gTimeCrtMS
                    0x0cef                  _gFileSlotOpen
                    0x0cf2                  _gFileArray
                    0x0dc4                  __fontHeight
                    0x0dc6                  __fontLastChar
                    0x0dc8                  __fontFirstChar
                    0x0dca                  __font
                    0x0dcc                  __fontOrientation
                    0x0dce                  __cursorY
                    0x0dd0                  __cursorX
                    0x0dd2                  __lineThickness
                    0x0dd4                  __lineType
                    0x0dd6                  _Couleur
                    0x0e00                  _IMG_pLoopCallbackFn
                    0x0e02                  _IMG_blAbortImageDecoding
                    0x0e03                  _IMG_bAlignCenter
                    0x0e04                  _IMG_bDownScalingFactor
                    0x0e06                  _IMG_wImageHeight
                    0x0e08                  _IMG_wImageWidth
                    0x0e0a                  _IMG_wHeight
                    0x0e0c                  _IMG_wWidth
                    0x0e0e                  _IMG_wStartY
                    0x0e10                  _IMG_wStartX
                    0x0e12                  __line_mem_pitch
                    0x0e16                  __visualPage
                    0x0e17                  __activePage
                    0x0e18                  __clipBottom
                    0x0e1a                  __clipRight
                    0x0e1c                  __clipTop
                    0x0e1e                  __clipLeft
                    0x0e20                  __clipRgn
                    0x0e22                  __color
                    0x0e24                  _cwdptr
                    0x0e26                  _recache
                    0x0e27                  _gBufferZeroed
                    0x0e28                  _nextClusterIsLast
                    0x0e29                  _gNeedDataWrite
                    0x0e2a                  _gLastDataSectorRead
                    0x0e2e                  _gBufferOwner
                    0x0e30                  _gNeedFATWrite
                    0x0e32                  _gLastFATSectorRead
                    0x0e36                  _MDD_SDSPI_finalLBA
                    0x0e3a                  _Counter
                    0x0e3e                  __gpioStatus
                    0x0ec8                  __Tls_setup__Randseed
                    0x0eca                  __Randseed
                    0x0ece                  __Tls_setup__Randinit
                    0x0ed0                  __Randinit

External Symbols in Data Memory (by name):

                    0x0dd6                  _Couleur
                    0x0e3a                  _Counter
                    0x0cde                  _FSerrno
                    0x0ce0                  _FatRootDirClusterValue
                    0x0e03                  _IMG_bAlignCenter
                    0x0e04                  _IMG_bDownScalingFactor
                    0x0e02                  _IMG_blAbortImageDecoding
                    0x0e00                  _IMG_pLoopCallbackFn
                    0x0e0a                  _IMG_wHeight
                    0x0e06                  _IMG_wImageHeight
                    0x0e08                  _IMG_wImageWidth
                    0x0e10                  _IMG_wStartX
                    0x0e0e                  _IMG_wStartY
                    0x0e0c                  _IMG_wWidth
                    0x0e36                  _MDD_SDSPI_finalLBA
                    0x0cda                  _TempClusterCalc
                    0x0ed0                  __Randinit
                    0x0eca                  __Randseed
                    0x0ece                  __Tls_setup__Randinit
                    0x0ec8                  __Tls_setup__Randseed
                    0x0e17                  __activePage
                    0x0e18                  __clipBottom
                    0x0e1e                  __clipLeft
                    0x0e20                  __clipRgn
                    0x0e1a                  __clipRight
                    0x0e1c                  __clipTop
                    0x0e22                  __color
                    0x0dd0                  __cursorX
                    0x0dce                  __cursorY
                    0x0dca                  __font
                    0x0dc8                  __fontFirstChar
                    0x0dc4                  __fontHeight
                    0x0dc6                  __fontLastChar
                    0x0dcc                  __fontOrientation
                    0x0e3e                  __gpioStatus
                    0x0dd2                  __lineThickness
                    0x0dd4                  __lineType
                    0x0e12                  __line_mem_pitch
                    0x0e16                  __visualPage
                    0x0c36                  _cwd
                    0x0e24                  _cwdptr
                    0x0c00                  _defaultArray
                    0x0c0a                  _defaultString
                    0x0cd8                  _dirCleared
                    0x0e2e                  _gBufferOwner
                    0x0e27                  _gBufferZeroed
                    0x0a00                  _gDataBuffer
                    0x0c18                  _gDiskData
                    0x0800                  _gFATBuffer
                    0x0cf2                  _gFileArray
                    0x0cef                  _gFileSlotOpen
                    0x0c6c                  _gFileTemp
                    0x0e2a                  _gLastDataSectorRead
                    0x0e32                  _gLastFATSectorRead
                    0x0e29                  _gNeedDataWrite
                    0x0e30                  _gNeedFATWrite
                    0x0ce8                  _gTimeAccDate
                    0x0cea                  _gTimeCrtDate
                    0x0cee                  _gTimeCrtMS
                    0x0cec                  _gTimeCrtTime
                    0x0ce4                  _gTimeWrtDate
                    0x0ce6                  _gTimeWrtTime
                    0x0e28                  _nextClusterIsLast
                    0x0e26                  _recache
                    0x0ca2                  _tempCWDobj

External Symbols in Program Memory (by address):

                  0x000200                  __resetPRI
                  0x00021e                  __psv_init
                  0x00022e                  __data_init
                  0x00028c                  _rand
                  0x000336                  _srand
                  0x000358                  _memset
                  0x000366                  _strncpy
                  0x00038c                  _toupper
                  0x00039a                  _tolower
                  0x0003a8                  _strlen
                  0x0003b6                  _strcpy
                  0x0003c6                  _strchr
                  0x0003d8                  ___floatsisf
                  0x00042e                  ___mulsf3
                  0x000496                  ___subsf3
                  0x000498                  ___addsf3
                  0x000552                  ___fixsfsi
                  0x000594                  ___modsi3
                  0x0005b2                  ___divsi3
                  0x0005d0                  ___udivsi3
                  0x0005f0                  ___umodsi3
                  0x0005f6                  __fpack
                  0x000642                  __funpack2
                  0x000652                  __fPropagateNaN
                  0x000664                  __fbopExit
                  0x00066c                  __fbopReturnNaN
                  0x000672                  __funpack
                  0x00069c                  ___mulsi3
                  0x0006a8                  _L1191258975
                  0x001c28                  _GOLFontDefault
                  0x001c2c                  _face
                  0x001c74                  _pz
                  0x001c84                  _py
                  0x001c94                  _px
                  0x001ca4                  _co
                  0x002244                  _si
                  0x002998                  _sdmmc_cmdtable
                  0x002a5a                  _Cluster2Sector
                  0x002aae                  _ReadByte
                  0x002ab4                  _LoadMBR
                  0x002bd2                  _ReadWord
                  0x002bde                  _ReadDWord
                  0x002c02                  _LoadBootSector
                  0x002d4a                  _DISKmount
                  0x002d82                  _FSInit
                  0x002dfa                  _GetFullClusterNumber
                  0x002e0e                  _flushData
                  0x002e3a                  _FSCreateMBR
                  0x002f8e                  _FSformat
                  0x00347e                  _Write_File_Entry
                  0x0034d2                  _WriteFAT
                  0x0036b6                  _ReadFAT
                  0x003882                  _Cache_File_Entry
                  0x0039d8                  _FILEget_next_cluster
                  0x003aa2                  _FAT_erase_cluster_chain
                  0x003b5c                  _LoadDirAttrib
                  0x003ba2                  _CacheTime
                  0x003c36                  _PopulateEntries
                  0x003cdc                  _FATfindEmptyCluster
                  0x003d96                  _EraseCluster
                  0x003df8                  _FILECreateHeadCluster
                  0x003e5e                  _CreateFirstCluster
                  0x003e9c                  _FILEallocate_new_cluster
                  0x003f0c                  _FindEmptyEntries
                  0x003f84                  _CreateFileEntry
                  0x003fd4                  _FSfclose
                  0x004070                  _Fill_File_Object
                  0x00412a                  _FILEopen
                  0x0041e8                  _FILEfind
                  0x00431c                  _FILEerase
                  0x004396                  _FileObjectCopy
                  0x0043a4                  _FSfseek
                  0x0044f0                  _FSftell
                  0x0044f8                  _FSrewind
                  0x00451c                  _FSerror
                  0x004522                  _FSattrib
                  0x00458a                  _FSfwrite
                  0x004758                  _FSfeof
                  0x004770                  _FSfread
                  0x0048ca                  _ValidateChars
                  0x004978                  _FormatFileName
                  0x004a14                  _FSremove
                  0x004aa2                  _FSfopen
                  0x004c80                  _FSrename
                  0x004d76                  _FormatDirName
                  0x004e12                  _chdirhelper
                  0x005046                  _FSchdir
                  0x00504e                  _GetPreviousEntry
                  0x005138                  _FSgetcwd
                  0x00538a                  _writeDotEntries
                  0x00543a                  _CreateDIR
                  0x005500                  _mkdirhelper
                  0x00571a                  _FSmkdir
                  0x005722                  _eraseDir
                  0x00578a                  _rmdirhelper
                  0x005a9e                  _FSrmdir
                  0x005aa8                  _FindFirst
                  0x005bfc                  _FindNext
                  0x005ed8                  _JPEG_bDecode
                  0x006e54                  _BDEC_vResetData
                  0x006e76                  _BDEC_bReadHeader
                  0x007034                  _BMP_bDecode
                  0x007cf8                  _DelayMs
                  0x007d0e                  _SetAddress
                  0x007d54                  _SetRegB
                  0x007dac                  _GetReg
                  0x007e2c                  _GetRegW
                  0x007e44                  _SetRegW
                  0x007e58                  _SetRegL
                  0x007e76                  _GetRegL
                  0x007e96                  _GPIO_SPENA
                  0x007ea8                  _GPIO_SPCLK
                  0x007eba                  _GPIO_SPDAT
                  0x007ecc                  _GPIO_SPRESET
                  0x007ede                  _PutPixel
                  0x007f58                  _GetPixel
                  0x007fca                  _Bar
                  0x00806c                  _ClearDevice
                  0x0080aa                  _PutImage1BPP
                  0x0081d0                  _PutImage4BPP
                  0x0082ec                  _PutImage8BPP
                  0x0083fc                  _PutImage16BPP
                  0x0084de                  _PutImage
                  0x008548                  _SPI_Write
                  0x008570                  _SPI_SetReg
                  0x0085a2                  _ResetDevice
                  0x00878a                  _ssd1928_FloatWndInit
                  0x00880a                  _ssd1928_FloatWndEnable
                  0x008826                  _ssd1928_MainWndInit
                  0x008884                  _ssd1928_FocusWnd
                  0x0088b2                  _ssd1928_MainWndEnable
                  0x0088ce                  _InitGraph
                  0x0088f8                  _Arc
                  0x008c4e                  _Line
                  0x008daa                  _Bevel
                  0x008f6c                  _FillBevel
                  0x009058                  _DrawPoly
                  0x00908c                  _SetFont
                  0x0090a4                  _OutChar
                  0x009180                  _OutText
                  0x0091a0                  _OutTextXY
                  0x0091ba                  _GetTextWidth
                  0x0091f0                  _GetTextHeight
                  0x009200                  _GetImageWidth
                  0x009220                  _GetImageHeight
                  0x009240                  _PixelOutput
                  0x009288                  _Obj3D
                  0x00945c                  _main
                  0x0099e4                  _jpeg_idct_islow
                  0x00a0f0                  _camVideoPreview
                  0x00a16c                  _camVideoStill
                  0x00a188                  _camCmdWr
                  0x00a1b2                  _camRegRd
                  0x00a1ea                  _camHwInit
                  0x00a4e2                  _camInit
                  0x00a53e                  _MDD_SDSPI_MediaDetect
                  0x00a546                  _MDD_SDSPI_ReadSectorSize
                  0x00a548                  _MDD_SDSPI_ReadCapacity
                  0x00a54e                  _MDD_SDSPI_InitIO
                  0x00a558                  _CloseSPIM
                  0x00a55c                  _MDD_SDSPI_ShutdownMedia
                  0x00a562                  _WriteSPIM
                  0x00a570                  _MDD_SDSPI_ReadMedia
                  0x00a580                  _SendMMCCmd
                  0x00a650                  _MDD_SDSPI_SectorRead
                  0x00a6e2                  _MDD_SDSPI_SectorWrite
                  0x00a768                  _MDD_SDSPI_WriteProtectState
                  0x00a770                  _Delayms
                  0x00a790                  _OpenSPIM
                  0x00a7a6                  _MDD_SDSPI_MediaInitialize
                  0x00a84e                  _ImageDecoderInit
                  0x00a862                  _ImageLoopCallbackRegister
                  0x00a866                  _ImageDecode
                  0x00a8a2                  _IMG_vSetboundaries
                  0x00a916                  _ssd1928_I2C_Init
                  0x00a92e                  _ssd1928_I2C_Wait
                  0x00a952                  _ssd1928_I2C_Ctl
                  0x00a966                  _ssd1928_I2C_Write
                  0x00a96c                  _ssd1928_I2C_Read
                  0x00aa2a                  __DefaultInterrupt

External Symbols in Program Memory (by name):

                  0x0088f8                  _Arc
                  0x006e76                  _BDEC_bReadHeader
                  0x006e54                  _BDEC_vResetData
                  0x007034                  _BMP_bDecode
                  0x007fca                  _Bar
                  0x008daa                  _Bevel
                  0x003ba2                  _CacheTime
                  0x003882                  _Cache_File_Entry
                  0x00806c                  _ClearDevice
                  0x00a558                  _CloseSPIM
                  0x002a5a                  _Cluster2Sector
                  0x00543a                  _CreateDIR
                  0x003f84                  _CreateFileEntry
                  0x003e5e                  _CreateFirstCluster
                  0x002d4a                  _DISKmount
                  0x007cf8                  _DelayMs
                  0x00a770                  _Delayms
                  0x009058                  _DrawPoly
                  0x003d96                  _EraseCluster
                  0x003aa2                  _FAT_erase_cluster_chain
                  0x003cdc                  _FATfindEmptyCluster
                  0x003df8                  _FILECreateHeadCluster
                  0x003e9c                  _FILEallocate_new_cluster
                  0x00431c                  _FILEerase
                  0x0041e8                  _FILEfind
                  0x0039d8                  _FILEget_next_cluster
                  0x00412a                  _FILEopen
                  0x002e3a                  _FSCreateMBR
                  0x002d82                  _FSInit
                  0x004522                  _FSattrib
                  0x005046                  _FSchdir
                  0x00451c                  _FSerror
                  0x003fd4                  _FSfclose
                  0x004758                  _FSfeof
                  0x004aa2                  _FSfopen
                  0x002f8e                  _FSformat
                  0x004770                  _FSfread
                  0x0043a4                  _FSfseek
                  0x0044f0                  _FSftell
                  0x00458a                  _FSfwrite
                  0x005138                  _FSgetcwd
                  0x00571a                  _FSmkdir
                  0x004a14                  _FSremove
                  0x004c80                  _FSrename
                  0x0044f8                  _FSrewind
                  0x005a9e                  _FSrmdir
                  0x004396                  _FileObjectCopy
                  0x008f6c                  _FillBevel
                  0x004070                  _Fill_File_Object
                  0x003f0c                  _FindEmptyEntries
                  0x005aa8                  _FindFirst
                  0x005bfc                  _FindNext
                  0x004d76                  _FormatDirName
                  0x004978                  _FormatFileName
                  0x001c28                  _GOLFontDefault
                  0x007ea8                  _GPIO_SPCLK
                  0x007eba                  _GPIO_SPDAT
                  0x007e96                  _GPIO_SPENA
                  0x007ecc                  _GPIO_SPRESET
                  0x002dfa                  _GetFullClusterNumber
                  0x009220                  _GetImageHeight
                  0x009200                  _GetImageWidth
                  0x007f58                  _GetPixel
                  0x00504e                  _GetPreviousEntry
                  0x007dac                  _GetReg
                  0x007e76                  _GetRegL
                  0x007e2c                  _GetRegW
                  0x0091f0                  _GetTextHeight
                  0x0091ba                  _GetTextWidth
                  0x00a8a2                  _IMG_vSetboundaries
                  0x00a866                  _ImageDecode
                  0x00a84e                  _ImageDecoderInit
                  0x00a862                  _ImageLoopCallbackRegister
                  0x0088ce                  _InitGraph
                  0x005ed8                  _JPEG_bDecode
                  0x0006a8                  _L1191258975
                  0x008c4e                  _Line
                  0x002c02                  _LoadBootSector
                  0x003b5c                  _LoadDirAttrib
                  0x002ab4                  _LoadMBR
                  0x00a54e                  _MDD_SDSPI_InitIO
                  0x00a53e                  _MDD_SDSPI_MediaDetect
                  0x00a7a6                  _MDD_SDSPI_MediaInitialize
                  0x00a548                  _MDD_SDSPI_ReadCapacity
                  0x00a570                  _MDD_SDSPI_ReadMedia
                  0x00a546                  _MDD_SDSPI_ReadSectorSize
                  0x00a650                  _MDD_SDSPI_SectorRead
                  0x00a6e2                  _MDD_SDSPI_SectorWrite
                  0x00a55c                  _MDD_SDSPI_ShutdownMedia
                  0x00a768                  _MDD_SDSPI_WriteProtectState
                  0x009288                  _Obj3D
                  0x00a790                  _OpenSPIM
                  0x0090a4                  _OutChar
                  0x009180                  _OutText
                  0x0091a0                  _OutTextXY
                  0x009240                  _PixelOutput
                  0x003c36                  _PopulateEntries
                  0x0084de                  _PutImage
                  0x0083fc                  _PutImage16BPP
                  0x0080aa                  _PutImage1BPP
                  0x0081d0                  _PutImage4BPP
                  0x0082ec                  _PutImage8BPP
                  0x007ede                  _PutPixel
                  0x002aae                  _ReadByte
                  0x002bde                  _ReadDWord
                  0x0036b6                  _ReadFAT
                  0x002bd2                  _ReadWord
                  0x0085a2                  _ResetDevice
                  0x008570                  _SPI_SetReg
                  0x008548                  _SPI_Write
                  0x00a580                  _SendMMCCmd
                  0x007d0e                  _SetAddress
                  0x00908c                  _SetFont
                  0x007d54                  _SetRegB
                  0x007e58                  _SetRegL
                  0x007e44                  _SetRegW
                  0x0048ca                  _ValidateChars
                  0x0034d2                  _WriteFAT
                  0x00a562                  _WriteSPIM
                  0x00347e                  _Write_File_Entry
                  0x00aa2a                  __DefaultInterrupt
                  0x000498                  ___addsf3
                  0x0005b2                  ___divsi3
                  0x000552                  ___fixsfsi
                  0x0003d8                  ___floatsisf
                  0x000594                  ___modsi3
                  0x00042e                  ___mulsf3
                  0x00069c                  ___mulsi3
                  0x000496                  ___subsf3
                  0x0005d0                  ___udivsi3
                  0x0005f0                  ___umodsi3
                  0x00022e                  __data_init
                  0x000652                  __fPropagateNaN
                  0x000664                  __fbopExit
                  0x00066c                  __fbopReturnNaN
                  0x0005f6                  __fpack
                  0x000672                  __funpack
                  0x000642                  __funpack2
                  0x00021e                  __psv_init
                  0x000200                  __resetPRI
                  0x00a188                  _camCmdWr
                  0x00a1ea                  _camHwInit
                  0x00a4e2                  _camInit
                  0x00a1b2                  _camRegRd
                  0x00a0f0                  _camVideoPreview
                  0x00a16c                  _camVideoStill
                  0x004e12                  _chdirhelper
                  0x001ca4                  _co
                  0x005722                  _eraseDir
                  0x001c2c                  _face
                  0x002e0e                  _flushData
                  0x0099e4                  _jpeg_idct_islow
                  0x00945c                  _main
                  0x000358                  _memset
                  0x005500                  _mkdirhelper
                  0x001c94                  _px
                  0x001c84                  _py
                  0x001c74                  _pz
                  0x00028c                  _rand
                  0x00578a                  _rmdirhelper
                  0x002998                  _sdmmc_cmdtable
                  0x002244                  _si
                  0x000336                  _srand
                  0x00880a                  _ssd1928_FloatWndEnable
                  0x00878a                  _ssd1928_FloatWndInit
                  0x008884                  _ssd1928_FocusWnd
                  0x00a952                  _ssd1928_I2C_Ctl
                  0x00a916                  _ssd1928_I2C_Init
                  0x00a96c                  _ssd1928_I2C_Read
                  0x00a92e                  _ssd1928_I2C_Wait
                  0x00a966                  _ssd1928_I2C_Write
                  0x0088b2                  _ssd1928_MainWndEnable
                  0x008826                  _ssd1928_MainWndInit
                  0x0003c6                  _strchr
                  0x0003b6                  _strcpy
                  0x0003a8                  _strlen
                  0x000366                  _strncpy
                  0x00039a                  _tolower
                  0x00038c                  _toupper
                  0x00538a                  _writeDotEntries

Memory Configuration

Name             Origin             Length             Attributes
data             0x000800           0x004000           a !xr
reset            0x000000           0x000004  
ivt              0x000004           0x0000fc  
aivt             0x000104           0x0000fc  
program          0x000200           0x02a9f8           xr
config4          0x02abf8           0x000002  
config3          0x02abfa           0x000002  
config2          0x02abfc           0x000002  
config1          0x02abfe           0x000002  
*default*        0x000000           0xffffffff  

Linker script and memory map

LOAD Objects - Image Decoders Demo\Application.o
LOAD Objects - Image Decoders Demo\JpegDecoder.o
LOAD Objects - Image Decoders Demo\BmpDecoder.o
LOAD Objects - Image Decoders Demo\GifDecoder.o
LOAD Objects - Image Decoders Demo\ImageDecoder.o
LOAD Objects - Image Decoders Demo\jidctint.o
LOAD Objects - Image Decoders Demo\Primitive.o
LOAD Objects - Image Decoders Demo\GOLFontDefault.o
LOAD Objects - Image Decoders Demo\DisplayDriver.o
LOAD Objects - Image Decoders Demo\SD-SPI.o
LOAD Objects - Image Decoders Demo\FSIO.o
LOAD Objects - Image Decoders Demo\ov9650.o
LOAD Objects - Image Decoders Demo\SSD1928_I2C.o
LOAD c:/program files/microchip/mplab c30/bin/bin/../../lib/PIC24F\libpPIC24Fxxx-coff.a
                    0x2abfa                  __CONFIG3 = 0x2abfa
                    0x2abfc                  __CONFIG2 = 0x2abfc
                    0x2abfe                  __CONFIG1 = 0x2abfe
                    0x0004                  __IVT_BASE = 0x4
                    0x0104                  __AIVT_BASE = 0x104
                    0x0800                  __DATA_BASE = 0x800
                    0x0200                  __CODE_BASE = 0x200

.reset            0x000000          0x4
                  0x000000          0x2 SHORT 0x200 <code 337> (__reset)
                  0x000001          0x2 SHORT 0x4
                  0x000002          0x2 SHORT 0x0 ((<code 337> (__reset) >> 0x10) & 0x7f)
                  0x000003          0x2 SHORT 0x0

.text             0x000200        0x4a8
 *(.init)
 .init            0x000200         0x88 c:/program files/microchip/mplab c30/bin/bin/../../lib\libpic30-coff.a(crt0.o)
                  0x000200                  _resetPRI
                  0x000200                  _reset
                  0x00021e                  _psv_init
                  0x00022e                  _data_init
 *(.user_init)
 *(.handle)
 .handle          0x000288          0x4 jump_table
 *(.libc)
 .libc            0x00028c         0xaa c:/program files/microchip/mplab c30/bin/bin/../../lib\libc-coff.a(rand.o)
                  0x00028c                  rand
 .libc            0x000336         0x22 c:/program files/microchip/mplab c30/bin/bin/../../lib\libc-coff.a(srand.o)
                  0x000336                  srand
 .libc            0x000358          0xe c:/program files/microchip/mplab c30/bin/bin/../../lib\libc-coff.a(memset.o)
                  0x000358                  memset
 .libc            0x000366         0x26 c:/program files/microchip/mplab c30/bin/bin/../../lib\libc-coff.a(strncpy.o)
                  0x000366                  strncpy
 .libc            0x00038c          0xe c:/program files/microchip/mplab c30/bin/bin/../../lib\libc-coff.a(toupper.os)
                  0x00038c                  toupper
 .libc            0x00039a          0xe c:/program files/microchip/mplab c30/bin/bin/../../lib\libc-coff.a(tolower.os)
                  0x00039a                  tolower
 .libc            0x0003a8          0xe c:/program files/microchip/mplab c30/bin/bin/../../lib\libc-coff.a(strlen.o)
                  0x0003a8                  strlen
 .libc            0x0003b6         0x10 c:/program files/microchip/mplab c30/bin/bin/../../lib\libc-coff.a(strcpy.o)
                  0x0003b6                  strcpy
 .libc            0x0003c6         0x12 c:/program files/microchip/mplab c30/bin/bin/../../lib\libc-coff.a(strchr.o)
                  0x0003c6                  strchr
 *(.libm)
 .libm            0x0003d8         0x56 c:/program files/microchip/mplab c30/bin/bin/../../lib\libm-coff.a(floatsisf.o)
                  0x0003d8                  __floatsisf
 .libm            0x00042e         0x68 c:/program files/microchip/mplab c30/bin/bin/../../lib\libm-coff.a(mulsf3.o)
                  0x00042e                  __mulsf3
 .libm            0x000496         0xbc c:/program files/microchip/mplab c30/bin/bin/../../lib\libm-coff.a(addsf3.o)
                  0x000496                  __subsf3
                  0x000498                  __addsf3
 .libm            0x000552         0x42 c:/program files/microchip/mplab c30/bin/bin/../../lib\libm-coff.a(fixsfsi.o)
                  0x000552                  __fixsfsi
 .libm            0x000594         0x1e c:/program files/microchip/mplab c30/bin/bin/../../lib\libm-coff.a(modsi3.o)
                  0x000594                  __modsi3
 .libm            0x0005b2         0x1e c:/program files/microchip/mplab c30/bin/bin/../../lib\libm-coff.a(divsi3.o)
                  0x0005b2                  __divsi3
 .libm            0x0005d0         0x20 c:/program files/microchip/mplab c30/bin/bin/../../lib\libm-coff.a(udivsi3.o)
                  0x0005d0                  __udivsi3
 .libm            0x0005f0          0x6 c:/program files/microchip/mplab c30/bin/bin/../../lib\libm-coff.a(umodsi3.o)
                  0x0005f0                  __umodsi3
 .libm            0x0005f6         0x4c c:/program files/microchip/mplab c30/bin/bin/../../lib\libm-coff.a(fpack.o)
                  0x0005f6                  _fpack
 .libm            0x000642         0x10 c:/program files/microchip/mplab c30/bin/bin/../../lib\libm-coff.a(funpack2.o)
                  0x000642                  _funpack2
 .libm            0x000652         0x20 c:/program files/microchip/mplab c30/bin/bin/../../lib\libm-coff.a(futil.o)
                  0x000652                  _fPropagateNaN
                  0x000664                  _fbopExit
                  0x00066c                  _fbopReturnNaN
 .libm            0x000672         0x2a c:/program files/microchip/mplab c30/bin/bin/../../lib\libm-coff.a(funpack.o)
                  0x000672                  _funpack
 .libm            0x00069c          0xc c:/program files/microchip/mplab c30/bin/bin/../../lib\libm-coff.a(mulsi3.o)
                  0x00069c                  __mulsi3
 *(.libdsp)
 *(.lib*)

__CONFIG3
 *(__CONFIG3.sec)

__CONFIG2         0x02abfc          0x2
 *(__CONFIG2.sec)
 __CONFIG2.sec    0x02abfc          0x2 Objects - Image Decoders Demo\Application.o

__CONFIG1         0x02abfe          0x2
 *(__CONFIG1.sec)
 __CONFIG1.sec    0x02abfe          0x2 Objects - Image Decoders Demo\Application.o

.comment
 *(.comment)

.debug_info
 *(.debug_info)
 *(.gnu.linkonce.wi.*)

.debug_abbrev
 *(.debug_abbrev)

.debug_line
 *(.debug_line)

.debug_frame
 *(.debug_frame)

.debug_str
 *(.debug_str)

.debug_loc
 *(.debug_loc)

.debug_macinfo
 *(.debug_macinfo)

.debug_pubnames
 *(.debug_pubnames)

.debug_ranges
 *(.debug_ranges)

.debug_aranges
 *(.debug_aranges)

.ivt              0x000004         0xfc
                  0x000004          0x4 LONG 0xaa2a DEFINED (__ReservedTrap0)?<code 337> (__ReservedTrap0):<code 337> (__DefaultInterrupt)
                  0x000006          0x4 LONG 0xaa2a DEFINED (__OscillatorFail)?<code 337> (__OscillatorFail):<code 337> (__DefaultInterrupt)
                  0x000008          0x4 LONG 0xaa2a DEFINED (__AddressError)?<code 337> (__AddressError):<code 337> (__DefaultInterrupt)
                  0x00000a          0x4 LONG 0xaa2a DEFINED (__StackError)?<code 337> (__StackError):<code 337> (__DefaultInterrupt)
                  0x00000c          0x4 LONG 0xaa2a DEFINED (__MathError)?<code 337> (__MathError):<code 337> (__DefaultInterrupt)
                  0x00000e          0x4 LONG 0xaa2a DEFINED (__ReservedTrap5)?<code 337> (__ReservedTrap5):<code 337> (__DefaultInterrupt)
                  0x000010          0x4 LONG 0xaa2a DEFINED (__ReservedTrap6)?<code 337> (__ReservedTrap6):<code 337> (__DefaultInterrupt)
                  0x000012          0x4 LONG 0xaa2a DEFINED (__ReservedTrap7)?<code 337> (__ReservedTrap7):<code 337> (__DefaultInterrupt)
                  0x000014          0x4 LONG 0xaa2a DEFINED (__INT0Interrupt)?<code 337> (__INT0Interrupt):<code 337> (__DefaultInterrupt)
                  0x000016          0x4 LONG 0xaa2a DEFINED (__IC1Interrupt)?<code 337> (__IC1Interrupt):<code 337> (__DefaultInterrupt)
                  0x000018          0x4 LONG 0xaa2a DEFINED (__OC1Interrupt)?<code 337> (__OC1Interrupt):<code 337> (__DefaultInterrupt)
                  0x00001a          0x4 LONG 0xaa2a DEFINED (__T1Interrupt)?<code 337> (__T1Interrupt):<code 337> (__DefaultInterrupt)
                  0x00001c          0x4 LONG 0xaa2a DEFINED (__Interrupt4)?<code 337> (__Interrupt4):<code 337> (__DefaultInterrupt)
                  0x00001e          0x4 LONG 0xaa2a DEFINED (__IC2Interrupt)?<code 337> (__IC2Interrupt):<code 337> (__DefaultInterrupt)
                  0x000020          0x4 LONG 0xaa2a DEFINED (__OC2Interrupt)?<code 337> (__OC2Interrupt):<code 337> (__DefaultInterrupt)
                  0x000022          0x4 LONG 0xaa2a DEFINED (__T2Interrupt)?<code 337> (__T2Interrupt):<code 337> (__DefaultInterrupt)
                  0x000024          0x4 LONG 0xaa2a DEFINED (__T3Interrupt)?<code 337> (__T3Interrupt):<code 337> (__DefaultInterrupt)
                  0x000026          0x4 LONG 0xaa2a DEFINED (__SPI1ErrInterrupt)?<code 337> (__SPI1ErrInterrupt):<code 337> (__DefaultInterrupt)
                  0x000028          0x4 LONG 0xaa2a DEFINED (__SPI1Interrupt)?<code 337> (__SPI1Interrupt):<code 337> (__DefaultInterrupt)
                  0x00002a          0x4 LONG 0xaa2a DEFINED (__U1RXInterrupt)?<code 337> (__U1RXInterrupt):<code 337> (__DefaultInterrupt)
                  0x00002c          0x4 LONG 0xaa2a DEFINED (__U1TXInterrupt)?<code 337> (__U1TXInterrupt):<code 337> (__DefaultInterrupt)
                  0x00002e          0x4 LONG 0xaa2a DEFINED (__ADC1Interrupt)?<code 337> (__ADC1Interrupt):<code 337> (__DefaultInterrupt)
                  0x000030          0x4 LONG 0xaa2a DEFINED (__Interrupt14)?<code 337> (__Interrupt14):<code 337> (__DefaultInterrupt)
                  0x000032          0x4 LONG 0xaa2a DEFINED (__Interrupt15)?<code 337> (__Interrupt15):<code 337> (__DefaultInterrupt)
                  0x000034          0x4 LONG 0xaa2a DEFINED (__SI2C1Interrupt)?<code 337> (__SI2C1Interrupt):<code 337> (__DefaultInterrupt)
                  0x000036          0x4 LONG 0xaa2a DEFINED (__MI2C1Interrupt)?<code 337> (__MI2C1Interrupt):<code 337> (__DefaultInterrupt)
                  0x000038          0x4 LONG 0xaa2a DEFINED (__CompInterrupt)?<code 337> (__CompInterrupt):<code 337> (__DefaultInterrupt)
                  0x00003a          0x4 LONG 0xaa2a DEFINED (__CNInterrupt)?<code 337> (__CNInterrupt):<code 337> (__DefaultInterrupt)
                  0x00003c          0x4 LONG 0xaa2a DEFINED (__INT1Interrupt)?<code 337> (__INT1Interrupt):<code 337> (__DefaultInterrupt)
                  0x00003e          0x4 LONG 0xaa2a DEFINED (__Interrupt21)?<code 337> (__Interrupt21):<code 337> (__DefaultInterrupt)
                  0x000040          0x4 LONG 0xaa2a DEFINED (__IC7Interrupt)?<code 337> (__IC7Interrupt):<code 337> (__DefaultInterrupt)
                  0x000042          0x4 LONG 0xaa2a DEFINED (__IC8Interrupt)?<code 337> (__IC8Interrupt):<code 337> (__DefaultInterrupt)
                  0x000044          0x4 LONG 0xaa2a DEFINED (__Interrupt24)?<code 337> (__Interrupt24):<code 337> (__DefaultInterrupt)
                  0x000046          0x4 LONG 0xaa2a DEFINED (__OC3Interrupt)?<code 337> (__OC3Interrupt):<code 337> (__DefaultInterrupt)
                  0x000048          0x4 LONG 0xaa2a DEFINED (__OC4Interrupt)?<code 337> (__OC4Interrupt):<code 337> (__DefaultInterrupt)
                  0x00004a          0x4 LONG 0xaa2a DEFINED (__T4Interrupt)?<code 337> (__T4Interrupt):<code 337> (__DefaultInterrupt)
                  0x00004c          0x4 LONG 0xaa2a DEFINED (__T5Interrupt)?<code 337> (__T5Interrupt):<code 337> (__DefaultInterrupt)
                  0x00004e          0x4 LONG 0xaa2a DEFINED (__INT2Interrupt)?<code 337> (__INT2Interrupt):<code 337> (__DefaultInterrupt)
                  0x000050          0x4 LONG 0xaa2a DEFINED (__U2RXInterrupt)?<code 337> (__U2RXInterrupt):<code 337> (__DefaultInterrupt)
                  0x000052          0x4 LONG 0xaa2a DEFINED (__U2TXInterrupt)?<code 337> (__U2TXInterrupt):<code 337> (__DefaultInterrupt)
                  0x000054          0x4 LONG 0xaa2a DEFINED (__SPI2ErrInterrupt)?<code 337> (__SPI2ErrInterrupt):<code 337> (__DefaultInterrupt)
                  0x000056          0x4 LONG 0xaa2a DEFINED (__SPI2Interrupt)?<code 337> (__SPI2Interrupt):<code 337> (__DefaultInterrupt)
                  0x000058          0x4 LONG 0xaa2a DEFINED (__Interrupt34)?<code 337> (__Interrupt34):<code 337> (__DefaultInterrupt)
                  0x00005a          0x4 LONG 0xaa2a DEFINED (__Interrupt35)?<code 337> (__Interrupt35):<code 337> (__DefaultInterrupt)
                  0x00005c          0x4 LONG 0xaa2a DEFINED (__Interrupt36)?<code 337> (__Interrupt36):<code 337> (__DefaultInterrupt)
                  0x00005e          0x4 LONG 0xaa2a DEFINED (__IC3Interrupt)?<code 337> (__IC3Interrupt):<code 337> (__DefaultInterrupt)
                  0x000060          0x4 LONG 0xaa2a DEFINED (__IC4Interrupt)?<code 337> (__IC4Interrupt):<code 337> (__DefaultInterrupt)
                  0x000062          0x4 LONG 0xaa2a DEFINED (__IC5Interrupt)?<code 337> (__IC5Interrupt):<code 337> (__DefaultInterrupt)
                  0x000064          0x4 LONG 0xaa2a DEFINED (__IC6Interrupt)?<code 337> (__IC6Interrupt):<code 337> (__DefaultInterrupt)
                  0x000066          0x4 LONG 0xaa2a DEFINED (__OC5Interrupt)?<code 337> (__OC5Interrupt):<code 337> (__DefaultInterrupt)
                  0x000068          0x4 LONG 0xaa2a DEFINED (__OC6Interrupt)?<code 337> (__OC6Interrupt):<code 337> (__DefaultInterrupt)
                  0x00006a          0x4 LONG 0xaa2a DEFINED (__OC7Interrupt)?<code 337> (__OC7Interrupt):<code 337> (__DefaultInterrupt)
                  0x00006c          0x4 LONG 0xaa2a DEFINED (__OC8Interrupt)?<code 337> (__OC8Interrupt):<code 337> (__DefaultInterrupt)
                  0x00006e          0x4 LONG 0xaa2a DEFINED (__PMPInterrupt)?<code 337> (__PMPInterrupt):<code 337> (__DefaultInterrupt)
                  0x000070          0x4 LONG 0xaa2a DEFINED (__Interrupt46)?<code 337> (__Interrupt46):<code 337> (__DefaultInterrupt)
                  0x000072          0x4 LONG 0xaa2a DEFINED (__Interrupt47)?<code 337> (__Interrupt47):<code 337> (__DefaultInterrupt)
                  0x000074          0x4 LONG 0xaa2a DEFINED (__Interrupt48)?<code 337> (__Interrupt48):<code 337> (__DefaultInterrupt)
                  0x000076          0x4 LONG 0xaa2a DEFINED (__SI2C2Interrupt)?<code 337> (__SI2C2Interrupt):<code 337> (__DefaultInterrupt)
                  0x000078          0x4 LONG 0xaa2a DEFINED (__MI2C2Interrupt)?<code 337> (__MI2C2Interrupt):<code 337> (__DefaultInterrupt)
                  0x00007a          0x4 LONG 0xaa2a DEFINED (__Interrupt51)?<code 337> (__Interrupt51):<code 337> (__DefaultInterrupt)
                  0x00007c          0x4 LONG 0xaa2a DEFINED (__Interrupt52)?<code 337> (__Interrupt52):<code 337> (__DefaultInterrupt)
                  0x00007e          0x4 LONG 0xaa2a DEFINED (__INT3Interrupt)?<code 337> (__INT3Interrupt):<code 337> (__DefaultInterrupt)
                  0x000080          0x4 LONG 0xaa2a DEFINED (__INT4Interrupt)?<code 337> (__INT4Interrupt):<code 337> (__DefaultInterrupt)
                  0x000082          0x4 LONG 0xaa2a DEFINED (__Interrupt55)?<code 337> (__Interrupt55):<code 337> (__DefaultInterrupt)
                  0x000084          0x4 LONG 0xaa2a DEFINED (__Interrupt56)?<code 337> (__Interrupt56):<code 337> (__DefaultInterrupt)
                  0x000086          0x4 LONG 0xaa2a DEFINED (__Interrupt57)?<code 337> (__Interrupt57):<code 337> (__DefaultInterrupt)
                  0x000088          0x4 LONG 0xaa2a DEFINED (__Interrupt58)?<code 337> (__Interrupt58):<code 337> (__DefaultInterrupt)
                  0x00008a          0x4 LONG 0xaa2a DEFINED (__Interrupt59)?<code 337> (__Interrupt59):<code 337> (__DefaultInterrupt)
                  0x00008c          0x4 LONG 0xaa2a DEFINED (__Interrupt60)?<code 337> (__Interrupt60):<code 337> (__DefaultInterrupt)
                  0x00008e          0x4 LONG 0xaa2a DEFINED (__Interrupt61)?<code 337> (__Interrupt61):<code 337> (__DefaultInterrupt)
                  0x000090          0x4 LONG 0xaa2a DEFINED (__RTCCInterrupt)?<code 337> (__RTCCInterrupt):<code 337> (__DefaultInterrupt)
                  0x000092          0x4 LONG 0xaa2a DEFINED (__Interrupt63)?<code 337> (__Interrupt63):<code 337> (__DefaultInterrupt)
                  0x000094          0x4 LONG 0xaa2a DEFINED (__Interrupt64)?<code 337> (__Interrupt64):<code 337> (__DefaultInterrupt)
                  0x000096          0x4 LONG 0xaa2a DEFINED (__U1ErrInterrupt)?<code 337> (__U1ErrInterrupt):<code 337> (__DefaultInterrupt)
                  0x000098          0x4 LONG 0xaa2a DEFINED (__U2ErrInterrupt)?<code 337> (__U2ErrInterrupt):<code 337> (__DefaultInterrupt)
                  0x00009a          0x4 LONG 0xaa2a DEFINED (__CRCInterrupt)?<code 337> (__CRCInterrupt):<code 337> (__DefaultInterrupt)
                  0x00009c          0x4 LONG 0xaa2a DEFINED (__Interrupt68)?<code 337> (__Interrupt68):<code 337> (__DefaultInterrupt)
                  0x00009e          0x4 LONG 0xaa2a DEFINED (__Interrupt69)?<code 337> (__Interrupt69):<code 337> (__DefaultInterrupt)
                  0x0000a0          0x4 LONG 0xaa2a DEFINED (__Interrupt70)?<code 337> (__Interrupt70):<code 337> (__DefaultInterrupt)
                  0x0000a2          0x4 LONG 0xaa2a DEFINED (__Interrupt71)?<code 337> (__Interrupt71):<code 337> (__DefaultInterrupt)
                  0x0000a4          0x4 LONG 0xaa2a DEFINED (__LVDInterrupt)?<code 337> (__LVDInterrupt):<code 337> (__DefaultInterrupt)
                  0x0000a6          0x4 LONG 0xaa2a DEFINED (__Interrupt73)?<code 337> (__Interrupt73):<code 337> (__DefaultInterrupt)
                  0x0000a8          0x4 LONG 0xaa2a DEFINED (__Interrupt74)?<code 337> (__Interrupt74):<code 337> (__DefaultInterrupt)
                  0x0000aa          0x4 LONG 0xaa2a DEFINED (__Interrupt75)?<code 337> (__Interrupt75):<code 337> (__DefaultInterrupt)
                  0x0000ac          0x4 LONG 0xaa2a DEFINED (__Interrupt76)?<code 337> (__Interrupt76):<code 337> (__DefaultInterrupt)
                  0x0000ae          0x4 LONG 0xaa2a DEFINED (__CTMUInterrupt)?<code 337> (__CTMUInterrupt):<code 337> (__DefaultInterrupt)
                  0x0000b0          0x4 LONG 0xaa2a DEFINED (__Interrupt78)?<code 337> (__Interrupt78):<code 337> (__DefaultInterrupt)
                  0x0000b2          0x4 LONG 0xaa2a DEFINED (__Interrupt79)?<code 337> (__Interrupt79):<code 337> (__DefaultInterrupt)
                  0x0000b4          0x4 LONG 0xaa2a DEFINED (__Interrupt80)?<code 337> (__Interrupt80):<code 337> (__DefaultInterrupt)
                  0x0000b6          0x4 LONG 0xaa2a DEFINED (__U3ErrInterrupt)?<code 337> (__U3ErrInterrupt):<code 337> (__DefaultInterrupt)
                  0x0000b8          0x4 LONG 0xaa2a DEFINED (__U3RXInterrupt)?<code 337> (__U3RXInterrupt):<code 337> (__DefaultInterrupt)
                  0x0000ba          0x4 LONG 0xaa2a DEFINED (__U3TXInterrupt)?<code 337> (__U3TXInterrupt):<code 337> (__DefaultInterrupt)
                  0x0000bc          0x4 LONG 0xaa2a DEFINED (__SI2C3Interrupt)?<code 337> (__SI2C3Interrupt):<code 337> (__DefaultInterrupt)
                  0x0000be          0x4 LONG 0xaa2a DEFINED (__MI2C3Interrupt)?<code 337> (__MI2C3Interrupt):<code 337> (__DefaultInterrupt)
                  0x0000c0          0x4 LONG 0xaa2a DEFINED (__Interrupt86)?<code 337> (__Interrupt86):<code 337> (__DefaultInterrupt)
                  0x0000c2          0x4 LONG 0xaa2a DEFINED (__U4ErrInterrupt)?<code 337> (__U4ErrInterrupt):<code 337> (__DefaultInterrupt)
                  0x0000c4          0x4 LONG 0xaa2a DEFINED (__U4RXInterrupt)?<code 337> (__U4RXInterrupt):<code 337> (__DefaultInterrupt)
                  0x0000c6          0x4 LONG 0xaa2a DEFINED (__U4TXInterrupt)?<code 337> (__U4TXInterrupt):<code 337> (__DefaultInterrupt)
                  0x0000c8          0x4 LONG 0xaa2a DEFINED (__SPI3ErrInterrupt)?<code 337> (__SPI3ErrInterrupt):<code 337> (__DefaultInterrupt)
                  0x0000ca          0x4 LONG 0xaa2a DEFINED (__SPI3Interrupt)?<code 337> (__SPI3Interrupt):<code 337> (__DefaultInterrupt)
                  0x0000cc          0x4 LONG 0xaa2a DEFINED (__OC9Interrupt)?<code 337> (__OC9Interrupt):<code 337> (__DefaultInterrupt)
                  0x0000ce          0x4 LONG 0xaa2a DEFINED (__IC9Interrupt)?<code 337> (__IC9Interrupt):<code 337> (__DefaultInterrupt)
                  0x0000d0          0x4 LONG 0xaa2a DEFINED (__Interrupt94)?<code 337> (__Interrupt94):<code 337> (__DefaultInterrupt)
                  0x0000d2          0x4 LONG 0xaa2a DEFINED (__Interrupt95)?<code 337> (__Interrupt95):<code 337> (__DefaultInterrupt)
                  0x0000d4          0x4 LONG 0xaa2a DEFINED (__Interrupt96)?<code 337> (__Interrupt96):<code 337> (__DefaultInterrupt)
                  0x0000d6          0x4 LONG 0xaa2a DEFINED (__Interrupt97)?<code 337> (__Interrupt97):<code 337> (__DefaultInterrupt)
                  0x0000d8          0x4 LONG 0xaa2a DEFINED (__Interrupt98)?<code 337> (__Interrupt98):<code 337> (__DefaultInterrupt)
                  0x0000da          0x4 LONG 0xaa2a DEFINED (__Interrupt99)?<code 337> (__Interrupt99):<code 337> (__DefaultInterrupt)
                  0x0000dc          0x4 LONG 0xaa2a DEFINED (__Interrupt100)?<code 337> (__Interrupt100):<code 337> (__DefaultInterrupt)
                  0x0000de          0x4 LONG 0xaa2a DEFINED (__Interrupt101)?<code 337> (__Interrupt101):<code 337> (__DefaultInterrupt)
                  0x0000e0          0x4 LONG 0xaa2a DEFINED (__Interrupt102)?<code 337> (__Interrupt102):<code 337> (__DefaultInterrupt)
                  0x0000e2          0x4 LONG 0xaa2a DEFINED (__Interrupt103)?<code 337> (__Interrupt103):<code 337> (__DefaultInterrupt)
                  0x0000e4          0x4 LONG 0xaa2a DEFINED (__Interrupt104)?<code 337> (__Interrupt104):<code 337> (__DefaultInterrupt)
                  0x0000e6          0x4 LONG 0xaa2a DEFINED (__Interrupt105)?<code 337> (__Interrupt105):<code 337> (__DefaultInterrupt)
                  0x0000e8          0x4 LONG 0xaa2a DEFINED (__Interrupt106)?<code 337> (__Interrupt106):<code 337> (__DefaultInterrupt)
                  0x0000ea          0x4 LONG 0xaa2a DEFINED (__Interrupt107)?<code 337> (__Interrupt107):<code 337> (__DefaultInterrupt)
                  0x0000ec          0x4 LONG 0xaa2a DEFINED (__Interrupt108)?<code 337> (__Interrupt108):<code 337> (__DefaultInterrupt)
                  0x0000ee          0x4 LONG 0xaa2a DEFINED (__Interrupt109)?<code 337> (__Interrupt109):<code 337> (__DefaultInterrupt)
                  0x0000f0          0x4 LONG 0xaa2a DEFINED (__Interrupt110)?<code 337> (__Interrupt110):<code 337> (__DefaultInterrupt)
                  0x0000f2          0x4 LONG 0xaa2a DEFINED (__Interrupt111)?<code 337> (__Interrupt111):<code 337> (__DefaultInterrupt)
                  0x0000f4          0x4 LONG 0xaa2a DEFINED (__Interrupt112)?<code 337> (__Interrupt112):<code 337> (__DefaultInterrupt)
                  0x0000f6          0x4 LONG 0xaa2a DEFINED (__Interrupt113)?<code 337> (__Interrupt113):<code 337> (__DefaultInterrupt)
                  0x0000f8          0x4 LONG 0xaa2a DEFINED (__Interrupt114)?<code 337> (__Interrupt114):<code 337> (__DefaultInterrupt)
                  0x0000fa          0x4 LONG 0xaa2a DEFINED (__Interrupt115)?<code 337> (__Interrupt115):<code 337> (__DefaultInterrupt)
                  0x0000fc          0x4 LONG 0xaa2a DEFINED (__Interrupt116)?<code 337> (__Interrupt116):<code 337> (__DefaultInterrupt)
                  0x0000fe          0x4 LONG 0xaa2a DEFINED (__Interrupt117)?<code 337> (__Interrupt117):<code 337> (__DefaultInterrupt)

.aivt             0x000104         0xfc
                  0x000104          0x4 LONG 0xaa2a DEFINED (__AltReservedTrap0)?<code 337> (__AltReservedTrap0):DEFINED (__ReservedTrap0)?<code 337> (__ReservedTrap0):<code 337> (__DefaultInterrupt)
                  0x000106          0x4 LONG 0xaa2a DEFINED (__AltOscillatorFail)?<code 337> (__AltOscillatorFail):DEFINED (__OscillatorFail)?<code 337> (__OscillatorFail):<code 337> (__DefaultInterrupt)
                  0x000108          0x4 LONG 0xaa2a DEFINED (__AltAddressError)?<code 337> (__AltAddressError):DEFINED (__AddressError)?<code 337> (__AddressError):<code 337> (__DefaultInterrupt)
                  0x00010a          0x4 LONG 0xaa2a DEFINED (__AltStackError)?<code 337> (__AltStackError):DEFINED (__StackError)?<code 337> (__StackError):<code 337> (__DefaultInterrupt)
                  0x00010c          0x4 LONG 0xaa2a DEFINED (__AltMathError)?<code 337> (__AltMathError):DEFINED (__MathError)?<code 337> (__MathError):<code 337> (__DefaultInterrupt)
                  0x00010e          0x4 LONG 0xaa2a DEFINED (__AltReservedTrap5)?<code 337> (__AltReservedTrap5):DEFINED (__ReservedTrap5)?<code 337> (__ReservedTrap5):<code 337> (__DefaultInterrupt)
                  0x000110          0x4 LONG 0xaa2a DEFINED (__AltReservedTrap6)?<code 337> (__AltReservedTrap6):DEFINED (__ReservedTrap6)?<code 337> (__ReservedTrap6):<code 337> (__DefaultInterrupt)
                  0x000112          0x4 LONG 0xaa2a DEFINED (__AltReservedTrap7)?<code 337> (__AltReservedTrap7):DEFINED (__ReservedTrap7)?<code 337> (__ReservedTrap7):<code 337> (__DefaultInterrupt)
                  0x000114          0x4 LONG 0xaa2a DEFINED (__AltINT0Interrupt)?<code 337> (__AltINT0Interrupt):DEFINED (__INT0Interrupt)?<code 337> (__INT0Interrupt):<code 337> (__DefaultInterrupt)
                  0x000116          0x4 LONG 0xaa2a DEFINED (__AltIC1Interrupt)?<code 337> (__AltIC1Interrupt):DEFINED (__IC1Interrupt)?<code 337> (__IC1Interrupt):<code 337> (__DefaultInterrupt)
                  0x000118          0x4 LONG 0xaa2a DEFINED (__AltOC1Interrupt)?<code 337> (__AltOC1Interrupt):DEFINED (__OC1Interrupt)?<code 337> (__OC1Interrupt):<code 337> (__DefaultInterrupt)
                  0x00011a          0x4 LONG 0xaa2a DEFINED (__AltT1Interrupt)?<code 337> (__AltT1Interrupt):DEFINED (__T1Interrupt)?<code 337> (__T1Interrupt):<code 337> (__DefaultInterrupt)
                  0x00011c          0x4 LONG 0xaa2a DEFINED (__AltInterrupt4)?<code 337> (__AltInterrupt4):DEFINED (__Interrupt4)?<code 337> (__Interrupt4):<code 337> (__DefaultInterrupt)
                  0x00011e          0x4 LONG 0xaa2a DEFINED (__AltIC2Interrupt)?<code 337> (__AltIC2Interrupt):DEFINED (__IC2Interrupt)?<code 337> (__IC2Interrupt):<code 337> (__DefaultInterrupt)
                  0x000120          0x4 LONG 0xaa2a DEFINED (__AltOC2Interrupt)?<code 337> (__AltOC2Interrupt):DEFINED (__OC2Interrupt)?<code 337> (__OC2Interrupt):<code 337> (__DefaultInterrupt)
                  0x000122          0x4 LONG 0xaa2a DEFINED (__AltT2Interrupt)?<code 337> (__AltT2Interrupt):DEFINED (__T2Interrupt)?<code 337> (__T2Interrupt):<code 337> (__DefaultInterrupt)
                  0x000124          0x4 LONG 0xaa2a DEFINED (__AltT3Interrupt)?<code 337> (__AltT3Interrupt):DEFINED (__T3Interrupt)?<code 337> (__T3Interrupt):<code 337> (__DefaultInterrupt)
                  0x000126          0x4 LONG 0xaa2a DEFINED (__AltSPI1ErrInterrupt)?<code 337> (__AltSPI1ErrInterrupt):DEFINED (__SPI1ErrInterrupt)?<code 337> (__SPI1ErrInterrupt):<code 337> (__DefaultInterrupt)
                  0x000128          0x4 LONG 0xaa2a DEFINED (__AltSPI1Interrupt)?<code 337> (__AltSPI1Interrupt):DEFINED (__SPI1Interrupt)?<code 337> (__SPI1Interrupt):<code 337> (__DefaultInterrupt)
                  0x00012a          0x4 LONG 0xaa2a DEFINED (__AltU1RXInterrupt)?<code 337> (__AltU1RXInterrupt):DEFINED (__U1RXInterrupt)?<code 337> (__U1RXInterrupt):<code 337> (__DefaultInterrupt)
                  0x00012c          0x4 LONG 0xaa2a DEFINED (__AltU1TXInterrupt)?<code 337> (__AltU1TXInterrupt):DEFINED (__U1TXInterrupt)?<code 337> (__U1TXInterrupt):<code 337> (__DefaultInterrupt)
                  0x00012e          0x4 LONG 0xaa2a DEFINED (__AltADC1Interrupt)?<code 337> (__AltADC1Interrupt):DEFINED (__ADC1Interrupt)?<code 337> (__ADC1Interrupt):<code 337> (__DefaultInterrupt)
                  0x000130          0x4 LONG 0xaa2a DEFINED (__AltInterrupt14)?<code 337> (__AltInterrupt14):DEFINED (__Interrupt14)?<code 337> (__Interrupt14):<code 337> (__DefaultInterrupt)
                  0x000132          0x4 LONG 0xaa2a DEFINED (__AltInterrupt15)?<code 337> (__AltInterrupt15):DEFINED (__Interrupt15)?<code 337> (__Interrupt15):<code 337> (__DefaultInterrupt)
                  0x000134          0x4 LONG 0xaa2a DEFINED (__AltSI2C1Interrupt)?<code 337> (__AltSI2C1Interrupt):DEFINED (__SI2C1Interrupt)?<code 337> (__SI2C1Interrupt):<code 337> (__DefaultInterrupt)
                  0x000136          0x4 LONG 0xaa2a DEFINED (__AltMI2C1Interrupt)?<code 337> (__AltMI2C1Interrupt):DEFINED (__MI2C1Interrupt)?<code 337> (__MI2C1Interrupt):<code 337> (__DefaultInterrupt)
                  0x000138          0x4 LONG 0xaa2a DEFINED (__AltCompInterrupt)?<code 337> (__AltCompInterrupt):DEFINED (__CompInterrupt)?<code 337> (__CompInterrupt):<code 337> (__DefaultInterrupt)
                  0x00013a          0x4 LONG 0xaa2a DEFINED (__AltCNInterrupt)?<code 337> (__AltCNInterrupt):DEFINED (__CNInterrupt)?<code 337> (__CNInterrupt):<code 337> (__DefaultInterrupt)
                  0x00013c          0x4 LONG 0xaa2a DEFINED (__AltINT1Interrupt)?<code 337> (__AltINT1Interrupt):DEFINED (__INT1Interrupt)?<code 337> (__INT1Interrupt):<code 337> (__DefaultInterrupt)
                  0x00013e          0x4 LONG 0xaa2a DEFINED (__AltInterrupt21)?<code 337> (__AltInterrupt21):DEFINED (__Interrupt21)?<code 337> (__Interrupt21):<code 337> (__DefaultInterrupt)
                  0x000140          0x4 LONG 0xaa2a DEFINED (__AltIC7Interrupt)?<code 337> (__AltIC7Interrupt):DEFINED (__IC7Interrupt)?<code 337> (__IC7Interrupt):<code 337> (__DefaultInterrupt)
                  0x000142          0x4 LONG 0xaa2a DEFINED (__AltIC8Interrupt)?<code 337> (__AltIC8Interrupt):DEFINED (__IC8Interrupt)?<code 337> (__IC8Interrupt):<code 337> (__DefaultInterrupt)
                  0x000144          0x4 LONG 0xaa2a DEFINED (__AltInterrupt24)?<code 337> (__AltInterrupt24):DEFINED (__Interrupt24)?<code 337> (__Interrupt24):<code 337> (__DefaultInterrupt)
                  0x000146          0x4 LONG 0xaa2a DEFINED (__AltOC3Interrupt)?<code 337> (__AltOC3Interrupt):DEFINED (__OC3Interrupt)?<code 337> (__OC3Interrupt):<code 337> (__DefaultInterrupt)
                  0x000148          0x4 LONG 0xaa2a DEFINED (__AltOC4Interrupt)?<code 337> (__AltOC4Interrupt):DEFINED (__OC4Interrupt)?<code 337> (__OC4Interrupt):<code 337> (__DefaultInterrupt)
                  0x00014a          0x4 LONG 0xaa2a DEFINED (__AltT4Interrupt)?<code 337> (__AltT4Interrupt):DEFINED (__T4Interrupt)?<code 337> (__T4Interrupt):<code 337> (__DefaultInterrupt)
                  0x00014c          0x4 LONG 0xaa2a DEFINED (__AltT5Interrupt)?<code 337> (__AltT5Interrupt):DEFINED (__T5Interrupt)?<code 337> (__T5Interrupt):<code 337> (__DefaultInterrupt)
                  0x00014e          0x4 LONG 0xaa2a DEFINED (__AltINT2Interrupt)?<code 337> (__AltINT2Interrupt):DEFINED (__INT2Interrupt)?<code 337> (__INT2Interrupt):<code 337> (__DefaultInterrupt)
                  0x000150          0x4 LONG 0xaa2a DEFINED (__AltU2RXInterrupt)?<code 337> (__AltU2RXInterrupt):DEFINED (__U2RXInterrupt)?<code 337> (__U2RXInterrupt):<code 337> (__DefaultInterrupt)
                  0x000152          0x4 LONG 0xaa2a DEFINED (__AltU2TXInterrupt)?<code 337> (__AltU2TXInterrupt):DEFINED (__U2TXInterrupt)?<code 337> (__U2TXInterrupt):<code 337> (__DefaultInterrupt)
                  0x000154          0x4 LONG 0xaa2a DEFINED (__AltSPI2ErrInterrupt)?<code 337> (__AltSPI2ErrInterrupt):DEFINED (__SPI2ErrInterrupt)?<code 337> (__SPI2ErrInterrupt):<code 337> (__DefaultInterrupt)
                  0x000156          0x4 LONG 0xaa2a DEFINED (__AltSPI2Interrupt)?<code 337> (__AltSPI2Interrupt):DEFINED (__SPI2Interrupt)?<code 337> (__SPI2Interrupt):<code 337> (__DefaultInterrupt)
                  0x000158          0x4 LONG 0xaa2a DEFINED (__AltInterrupt34)?<code 337> (__AltInterrupt34):DEFINED (__Interrupt34)?<code 337> (__Interrupt34):<code 337> (__DefaultInterrupt)
                  0x00015a          0x4 LONG 0xaa2a DEFINED (__AltInterrupt35)?<code 337> (__AltInterrupt35):DEFINED (__Interrupt35)?<code 337> (__Interrupt35):<code 337> (__DefaultInterrupt)
                  0x00015c          0x4 LONG 0xaa2a DEFINED (__AltInterrupt36)?<code 337> (__AltInterrupt36):DEFINED (__Interrupt36)?<code 337> (__Interrupt36):<code 337> (__DefaultInterrupt)
                  0x00015e          0x4 LONG 0xaa2a DEFINED (__AltIC3Interrupt)?<code 337> (__AltIC3Interrupt):DEFINED (__IC3Interrupt)?<code 337> (__IC3Interrupt):<code 337> (__DefaultInterrupt)
                  0x000160          0x4 LONG 0xaa2a DEFINED (__AltIC4Interrupt)?<code 337> (__AltIC4Interrupt):DEFINED (__IC4Interrupt)?<code 337> (__IC4Interrupt):<code 337> (__DefaultInterrupt)
                  0x000162          0x4 LONG 0xaa2a DEFINED (__AltIC5Interrupt)?<code 337> (__AltIC5Interrupt):DEFINED (__IC5Interrupt)?<code 337> (__IC5Interrupt):<code 337> (__DefaultInterrupt)
                  0x000164          0x4 LONG 0xaa2a DEFINED (__AltIC6Interrupt)?<code 337> (__AltIC6Interrupt):DEFINED (__IC6Interrupt)?<code 337> (__IC6Interrupt):<code 337> (__DefaultInterrupt)
                  0x000166          0x4 LONG 0xaa2a DEFINED (__AltOC5Interrupt)?<code 337> (__AltOC5Interrupt):DEFINED (__OC5Interrupt)?<code 337> (__OC5Interrupt):<code 337> (__DefaultInterrupt)
                  0x000168          0x4 LONG 0xaa2a DEFINED (__AltOC6Interrupt)?<code 337> (__AltOC6Interrupt):DEFINED (__OC6Interrupt)?<code 337> (__OC6Interrupt):<code 337> (__DefaultInterrupt)
                  0x00016a          0x4 LONG 0xaa2a DEFINED (__AltOC7Interrupt)?<code 337> (__AltOC7Interrupt):DEFINED (__OC7Interrupt)?<code 337> (__OC7Interrupt):<code 337> (__DefaultInterrupt)
                  0x00016c          0x4 LONG 0xaa2a DEFINED (__AltOC8Interrupt)?<code 337> (__AltOC8Interrupt):DEFINED (__OC8Interrupt)?<code 337> (__OC8Interrupt):<code 337> (__DefaultInterrupt)
                  0x00016e          0x4 LONG 0xaa2a DEFINED (__AltPMPInterrupt)?<code 337> (__AltPMPInterrupt):DEFINED (__PMPInterrupt)?<code 337> (__PMPInterrupt):<code 337> (__DefaultInterrupt)
                  0x000170          0x4 LONG 0xaa2a DEFINED (__AltInterrupt46)?<code 337> (__AltInterrupt46):DEFINED (__Interrupt46)?<code 337> (__Interrupt46):<code 337> (__DefaultInterrupt)
                  0x000172          0x4 LONG 0xaa2a DEFINED (__AltInterrupt47)?<code 337> (__AltInterrupt47):DEFINED (__Interrupt47)?<code 337> (__Interrupt47):<code 337> (__DefaultInterrupt)
                  0x000174          0x4 LONG 0xaa2a DEFINED (__AltInterrupt48)?<code 337> (__AltInterrupt48):DEFINED (__Interrupt48)?<code 337> (__Interrupt48):<code 337> (__DefaultInterrupt)
                  0x000176          0x4 LONG 0xaa2a DEFINED (__AltSI2C2Interrupt)?<code 337> (__AltSI2C2Interrupt):DEFINED (__SI2C2Interrupt)?<code 337> (__SI2C2Interrupt):<code 337> (__DefaultInterrupt)
                  0x000178          0x4 LONG 0xaa2a DEFINED (__AltMI2C2Interrupt)?<code 337> (__AltMI2C2Interrupt):DEFINED (__MI2C2Interrupt)?<code 337> (__MI2C2Interrupt):<code 337> (__DefaultInterrupt)
                  0x00017a          0x4 LONG 0xaa2a DEFINED (__AltInterrupt51)?<code 337> (__AltInterrupt51):DEFINED (__Interrupt51)?<code 337> (__Interrupt51):<code 337> (__DefaultInterrupt)
                  0x00017c          0x4 LONG 0xaa2a DEFINED (__AltInterrupt52)?<code 337> (__AltInterrupt52):DEFINED (__Interrupt52)?<code 337> (__Interrupt52):<code 337> (__DefaultInterrupt)
                  0x00017e          0x4 LONG 0xaa2a DEFINED (__AltINT3Interrupt)?<code 337> (__AltINT3Interrupt):DEFINED (__INT3Interrupt)?<code 337> (__INT3Interrupt):<code 337> (__DefaultInterrupt)
                  0x000180          0x4 LONG 0xaa2a DEFINED (__AltINT4Interrupt)?<code 337> (__AltINT4Interrupt):DEFINED (__INT4Interrupt)?<code 337> (__INT4Interrupt):<code 337> (__DefaultInterrupt)
                  0x000182          0x4 LONG 0xaa2a DEFINED (__AltInterrupt55)?<code 337> (__AltInterrupt55):DEFINED (__Interrupt55)?<code 337> (__Interrupt55):<code 337> (__DefaultInterrupt)
                  0x000184          0x4 LONG 0xaa2a DEFINED (__AltInterrupt56)?<code 337> (__AltInterrupt56):DEFINED (__Interrupt56)?<code 337> (__Interrupt56):<code 337> (__DefaultInterrupt)
                  0x000186          0x4 LONG 0xaa2a DEFINED (__AltInterrupt57)?<code 337> (__AltInterrupt57):DEFINED (__Interrupt57)?<code 337> (__Interrupt57):<code 337> (__DefaultInterrupt)
                  0x000188          0x4 LONG 0xaa2a DEFINED (__AltInterrupt58)?<code 337> (__AltInterrupt58):DEFINED (__Interrupt58)?<code 337> (__Interrupt58):<code 337> (__DefaultInterrupt)
                  0x00018a          0x4 LONG 0xaa2a DEFINED (__AltInterrupt59)?<code 337> (__AltInterrupt59):DEFINED (__Interrupt59)?<code 337> (__Interrupt59):<code 337> (__DefaultInterrupt)
                  0x00018c          0x4 LONG 0xaa2a DEFINED (__AltInterrupt60)?<code 337> (__AltInterrupt60):DEFINED (__Interrupt60)?<code 337> (__Interrupt60):<code 337> (__DefaultInterrupt)
                  0x00018e          0x4 LONG 0xaa2a DEFINED (__AltInterrupt61)?<code 337> (__AltInterrupt61):DEFINED (__Interrupt61)?<code 337> (__Interrupt61):<code 337> (__DefaultInterrupt)
                  0x000190          0x4 LONG 0xaa2a DEFINED (__AltRTCCInterrupt)?<code 337> (__AltRTCCInterrupt):DEFINED (__RTCCInterrupt)?<code 337> (__RTCCInterrupt):<code 337> (__DefaultInterrupt)
                  0x000192          0x4 LONG 0xaa2a DEFINED (__AltInterrupt63)?<code 337> (__AltInterrupt63):DEFINED (__Interrupt63)?<code 337> (__Interrupt63):<code 337> (__DefaultInterrupt)
                  0x000194          0x4 LONG 0xaa2a DEFINED (__AltInterrupt64)?<code 337> (__AltInterrupt64):DEFINED (__Interrupt64)?<code 337> (__Interrupt64):<code 337> (__DefaultInterrupt)
                  0x000196          0x4 LONG 0xaa2a DEFINED (__AltU1ErrInterrupt)?<code 337> (__AltU1ErrInterrupt):DEFINED (__U1ErrInterrupt)?<code 337> (__U1ErrInterrupt):<code 337> (__DefaultInterrupt)
                  0x000198          0x4 LONG 0xaa2a DEFINED (__AltU2ErrInterrupt)?<code 337> (__AltU2ErrInterrupt):DEFINED (__U2ErrInterrupt)?<code 337> (__U2ErrInterrupt):<code 337> (__DefaultInterrupt)
                  0x00019a          0x4 LONG 0xaa2a DEFINED (__AltCRCInterrupt)?<code 337> (__AltCRCInterrupt):DEFINED (__CRCInterrupt)?<code 337> (__CRCInterrupt):<code 337> (__DefaultInterrupt)
                  0x00019c          0x4 LONG 0xaa2a DEFINED (__AltInterrupt68)?<code 337> (__AltInterrupt68):DEFINED (__Interrupt68)?<code 337> (__Interrupt68):<code 337> (__DefaultInterrupt)
                  0x00019e          0x4 LONG 0xaa2a DEFINED (__AltInterrupt69)?<code 337> (__AltInterrupt69):DEFINED (__Interrupt69)?<code 337> (__Interrupt69):<code 337> (__DefaultInterrupt)
                  0x0001a0          0x4 LONG 0xaa2a DEFINED (__AltInterrupt70)?<code 337> (__AltInterrupt70):DEFINED (__Interrupt70)?<code 337> (__Interrupt70):<code 337> (__DefaultInterrupt)
                  0x0001a2          0x4 LONG 0xaa2a DEFINED (__AltInterrupt71)?<code 337> (__AltInterrupt71):DEFINED (__Interrupt71)?<code 337> (__Interrupt71):<code 337> (__DefaultInterrupt)
                  0x0001a4          0x4 LONG 0xaa2a DEFINED (__AltLVDInterrupt)?<code 337> (__AltLVDInterrupt):DEFINED (__LVDInterrupt)?<code 337> (__LVDInterrupt):<code 337> (__DefaultInterrupt)
                  0x0001a6          0x4 LONG 0xaa2a DEFINED (__AltInterrupt73)?<code 337> (__AltInterrupt73):DEFINED (__Interrupt73)?<code 337> (__Interrupt73):<code 337> (__DefaultInterrupt)
                  0x0001a8          0x4 LONG 0xaa2a DEFINED (__AltInterrupt74)?<code 337> (__AltInterrupt74):DEFINED (__Interrupt74)?<code 337> (__Interrupt74):<code 337> (__DefaultInterrupt)
                  0x0001aa          0x4 LONG 0xaa2a DEFINED (__AltInterrupt75)?<code 337> (__AltInterrupt75):DEFINED (__Interrupt75)?<code 337> (__Interrupt75):<code 337> (__DefaultInterrupt)
                  0x0001ac          0x4 LONG 0xaa2a DEFINED (__AltInterrupt76)?<code 337> (__AltInterrupt76):DEFINED (__Interrupt76)?<code 337> (__Interrupt76):<code 337> (__DefaultInterrupt)
                  0x0001ae          0x4 LONG 0xaa2a DEFINED (__AltCTMUInterrupt)?<code 337> (__AltCTMUInterrupt):DEFINED (__CTMUInterrupt)?<code 337> (__CTMUInterrupt):<code 337> (__DefaultInterrupt)
                  0x0001b0          0x4 LONG 0xaa2a DEFINED (__AltInterrupt78)?<code 337> (__AltInterrupt78):DEFINED (__Interrupt78)?<code 337> (__Interrupt78):<code 337> (__DefaultInterrupt)
                  0x0001b2          0x4 LONG 0xaa2a DEFINED (__AltInterrupt79)?<code 337> (__AltInterrupt79):DEFINED (__Interrupt79)?<code 337> (__Interrupt79):<code 337> (__DefaultInterrupt)
                  0x0001b4          0x4 LONG 0xaa2a DEFINED (__AltInterrupt80)?<code 337> (__AltInterrupt80):DEFINED (__Interrupt80)?<code 337> (__Interrupt80):<code 337> (__DefaultInterrupt)
                  0x0001b6          0x4 LONG 0xaa2a DEFINED (__AltU3ErrInterrupt)?<code 337> (__AltU3ErrInterrupt):DEFINED (__U3ErrInterrupt)?<code 337> (__U3ErrInterrupt):<code 337> (__DefaultInterrupt)
                  0x0001b8          0x4 LONG 0xaa2a DEFINED (__AltU3RXInterrupt)?<code 337> (__AltU3RXInterrupt):DEFINED (__U3RXInterrupt)?<code 337> (__U3RXInterrupt):<code 337> (__DefaultInterrupt)
                  0x0001ba          0x4 LONG 0xaa2a DEFINED (__AltU3TXInterrupt)?<code 337> (__AltU3TXInterrupt):DEFINED (__U3TXInterrupt)?<code 337> (__U3TXInterrupt):<code 337> (__DefaultInterrupt)
                  0x0001bc          0x4 LONG 0xaa2a DEFINED (__AltSI2C3Interrupt)?<code 337> (__AltSI2C3Interrupt):DEFINED (__SI2C3Interrupt)?<code 337> (__SI2C3Interrupt):<code 337> (__DefaultInterrupt)
                  0x0001be          0x4 LONG 0xaa2a DEFINED (__AltMI2C3Interrupt)?<code 337> (__AltMI2C3Interrupt):DEFINED (__MI2C3Interrupt)?<code 337> (__MI2C3Interrupt):<code 337> (__DefaultInterrupt)
                  0x0001c0          0x4 LONG 0xaa2a DEFINED (__AltInterrupt86)?<code 337> (__AltInterrupt86):DEFINED (__Interrupt86)?<code 337> (__Interrupt86):<code 337> (__DefaultInterrupt)
                  0x0001c2          0x4 LONG 0xaa2a DEFINED (__AltU4ErrInterrupt)?<code 337> (__AltU4ErrInterrupt):DEFINED (__U4ErrInterrupt)?<code 337> (__U4ErrInterrupt):<code 337> (__DefaultInterrupt)
                  0x0001c4          0x4 LONG 0xaa2a DEFINED (__AltU4RXInterrupt)?<code 337> (__AltU4RXInterrupt):DEFINED (__U4RXInterrupt)?<code 337> (__U4RXInterrupt):<code 337> (__DefaultInterrupt)
                  0x0001c6          0x4 LONG 0xaa2a DEFINED (__AltU4TXInterrupt)?<code 337> (__AltU4TXInterrupt):DEFINED (__U4TXInterrupt)?<code 337> (__U4TXInterrupt):<code 337> (__DefaultInterrupt)
                  0x0001c8          0x4 LONG 0xaa2a DEFINED (__AltSPI3ErrInterrupt)?<code 337> (__AltSPI3ErrInterrupt):DEFINED (__SPI3ErrInterrupt)?<code 337> (__SPI3ErrInterrupt):<code 337> (__DefaultInterrupt)
                  0x0001ca          0x4 LONG 0xaa2a DEFINED (__AltSPI3Interrupt)?<code 337> (__AltSPI3Interrupt):DEFINED (__SPI3Interrupt)?<code 337> (__SPI3Interrupt):<code 337> (__DefaultInterrupt)
                  0x0001cc          0x4 LONG 0xaa2a DEFINED (__AltOC9Interrupt)?<code 337> (__AltOC9Interrupt):DEFINED (__OC9Interrupt)?<code 337> (__OC9Interrupt):<code 337> (__DefaultInterrupt)
                  0x0001ce          0x4 LONG 0xaa2a DEFINED (__AltIC9Interrupt)?<code 337> (__AltIC9Interrupt):DEFINED (__IC9Interrupt)?<code 337> (__IC9Interrupt):<code 337> (__DefaultInterrupt)
                  0x0001d0          0x4 LONG 0xaa2a DEFINED (__AltInterrupt94)?<code 337> (__AltInterrupt94):DEFINED (__Interrupt94)?<code 337> (__Interrupt94):<code 337> (__DefaultInterrupt)
                  0x0001d2          0x4 LONG 0xaa2a DEFINED (__AltInterrupt95)?<code 337> (__AltInterrupt95):DEFINED (__Interrupt95)?<code 337> (__Interrupt95):<code 337> (__DefaultInterrupt)
                  0x0001d4          0x4 LONG 0xaa2a DEFINED (__AltInterrupt96)?<code 337> (__AltInterrupt96):DEFINED (__Interrupt96)?<code 337> (__Interrupt96):<code 337> (__DefaultInterrupt)
                  0x0001d6          0x4 LONG 0xaa2a DEFINED (__AltInterrupt97)?<code 337> (__AltInterrupt97):DEFINED (__Interrupt97)?<code 337> (__Interrupt97):<code 337> (__DefaultInterrupt)
                  0x0001d8          0x4 LONG 0xaa2a DEFINED (__AltInterrupt98)?<code 337> (__AltInterrupt98):DEFINED (__Interrupt98)?<code 337> (__Interrupt98):<code 337> (__DefaultInterrupt)
                  0x0001da          0x4 LONG 0xaa2a DEFINED (__AltInterrupt99)?<code 337> (__AltInterrupt99):DEFINED (__Interrupt99)?<code 337> (__Interrupt99):<code 337> (__DefaultInterrupt)
                  0x0001dc          0x4 LONG 0xaa2a DEFINED (__AltInterrupt100)?<code 337> (__AltInterrupt100):DEFINED (__Interrupt100)?<code 337> (__Interrupt100):<code 337> (__DefaultInterrupt)
                  0x0001de          0x4 LONG 0xaa2a DEFINED (__AltInterrupt101)?<code 337> (__AltInterrupt101):DEFINED (__Interrupt101)?<code 337> (__Interrupt101):<code 337> (__DefaultInterrupt)
                  0x0001e0          0x4 LONG 0xaa2a DEFINED (__AltInterrupt102)?<code 337> (__AltInterrupt102):DEFINED (__Interrupt102)?<code 337> (__Interrupt102):<code 337> (__DefaultInterrupt)
                  0x0001e2          0x4 LONG 0xaa2a DEFINED (__AltInterrupt103)?<code 337> (__AltInterrupt103):DEFINED (__Interrupt103)?<code 337> (__Interrupt103):<code 337> (__DefaultInterrupt)
                  0x0001e4          0x4 LONG 0xaa2a DEFINED (__AltInterrupt104)?<code 337> (__AltInterrupt104):DEFINED (__Interrupt104)?<code 337> (__Interrupt104):<code 337> (__DefaultInterrupt)
                  0x0001e6          0x4 LONG 0xaa2a DEFINED (__AltInterrupt105)?<code 337> (__AltInterrupt105):DEFINED (__Interrupt105)?<code 337> (__Interrupt105):<code 337> (__DefaultInterrupt)
                  0x0001e8          0x4 LONG 0xaa2a DEFINED (__AltInterrupt106)?<code 337> (__AltInterrupt106):DEFINED (__Interrupt106)?<code 337> (__Interrupt106):<code 337> (__DefaultInterrupt)
                  0x0001ea          0x4 LONG 0xaa2a DEFINED (__AltInterrupt107)?<code 337> (__AltInterrupt107):DEFINED (__Interrupt107)?<code 337> (__Interrupt107):<code 337> (__DefaultInterrupt)
                  0x0001ec          0x4 LONG 0xaa2a DEFINED (__AltInterrupt108)?<code 337> (__AltInterrupt108):DEFINED (__Interrupt108)?<code 337> (__Interrupt108):<code 337> (__DefaultInterrupt)
                  0x0001ee          0x4 LONG 0xaa2a DEFINED (__AltInterrupt109)?<code 337> (__AltInterrupt109):DEFINED (__Interrupt109)?<code 337> (__Interrupt109):<code 337> (__DefaultInterrupt)
                  0x0001f0          0x4 LONG 0xaa2a DEFINED (__AltInterrupt110)?<code 337> (__AltInterrupt110):DEFINED (__Interrupt110)?<code 337> (__Interrupt110):<code 337> (__DefaultInterrupt)
                  0x0001f2          0x4 LONG 0xaa2a DEFINED (__AltInterrupt111)?<code 337> (__AltInterrupt111):DEFINED (__Interrupt111)?<code 337> (__Interrupt111):<code 337> (__DefaultInterrupt)
                  0x0001f4          0x4 LONG 0xaa2a DEFINED (__AltInterrupt112)?<code 337> (__AltInterrupt112):DEFINED (__Interrupt112)?<code 337> (__Interrupt112):<code 337> (__DefaultInterrupt)
                  0x0001f6          0x4 LONG 0xaa2a DEFINED (__AltInterrupt113)?<code 337> (__AltInterrupt113):DEFINED (__Interrupt113)?<code 337> (__Interrupt113):<code 337> (__DefaultInterrupt)
                  0x0001f8          0x4 LONG 0xaa2a DEFINED (__AltInterrupt114)?<code 337> (__AltInterrupt114):DEFINED (__Interrupt114)?<code 337> (__Interrupt114):<code 337> (__DefaultInterrupt)
                  0x0001fa          0x4 LONG 0xaa2a DEFINED (__AltInterrupt115)?<code 337> (__AltInterrupt115):DEFINED (__Interrupt115)?<code 337> (__Interrupt115):<code 337> (__DefaultInterrupt)
                  0x0001fc          0x4 LONG 0xaa2a DEFINED (__AltInterrupt116)?<code 337> (__AltInterrupt116):DEFINED (__Interrupt116)?<code 337> (__Interrupt116):<code 337> (__DefaultInterrupt)
                  0x0001fe          0x4 LONG 0xaa2a DEFINED (__AltInterrupt117)?<code 337> (__AltInterrupt117):DEFINED (__Interrupt117)?<code 337> (__Interrupt117):<code 337> (__DefaultInterrupt)
                    0x0000                  WREG0 = 0x0
                    0x0000                  _WREG0 = 0x0
                    0x0002                  WREG1 = 0x2
                    0x0002                  _WREG1 = 0x2
                    0x0004                  WREG2 = 0x4
                    0x0004                  _WREG2 = 0x4
                    0x0006                  WREG3 = 0x6
                    0x0006                  _WREG3 = 0x6
                    0x0008                  WREG4 = 0x8
                    0x0008                  _WREG4 = 0x8
                    0x000a                  WREG5 = 0xa
                    0x000a                  _WREG5 = 0xa
                    0x000c                  WREG6 = 0xc
                    0x000c                  _WREG6 = 0xc
                    0x000e                  WREG7 = 0xe
                    0x000e                  _WREG7 = 0xe
                    0x0010                  WREG8 = 0x10
                    0x0010                  _WREG8 = 0x10
                    0x0012                  WREG9 = 0x12
                    0x0012                  _WREG9 = 0x12
                    0x0014                  WREG10 = 0x14
                    0x0014                  _WREG10 = 0x14
                    0x0016                  WREG11 = 0x16
                    0x0016                  _WREG11 = 0x16
                    0x0018                  WREG12 = 0x18
                    0x0018                  _WREG12 = 0x18
                    0x001a                  WREG13 = 0x1a
                    0x001a                  _WREG13 = 0x1a
                    0x001c                  WREG14 = 0x1c
                    0x001c                  _WREG14 = 0x1c
                    0x001e                  WREG15 = 0x1e
                    0x001e                  _WREG15 = 0x1e
                    0x0020                  SPLIM = 0x20
                    0x0020                  _SPLIM = 0x20
                    0x002e                  PCL = 0x2e
                    0x002e                  _PCL = 0x2e
                    0x0030                  PCH = 0x30
                    0x0030                  _PCH = 0x30
                    0x0032                  TBLPAG = 0x32
                    0x0032                  _TBLPAG = 0x32
                    0x0034                  PSVPAG = 0x34
                    0x0034                  _PSVPAG = 0x34
                    0x0036                  RCOUNT = 0x36
                    0x0036                  _RCOUNT = 0x36
                    0x0042                  SR = 0x42
                    0x0042                  _SR = 0x42
                    0x0042                  _SRbits = 0x42
                    0x0044                  CORCON = 0x44
                    0x0044                  _CORCON = 0x44
                    0x0044                  _CORCONbits = 0x44
                    0x0052                  DISICNT = 0x52
                    0x0052                  _DISICNT = 0x52
                    0x0054                  CNPD1 = 0x54
                    0x0054                  _CNPD1 = 0x54
                    0x0054                  _CNPD1bits = 0x54
                    0x0056                  CNPD2 = 0x56
                    0x0056                  _CNPD2 = 0x56
                    0x0056                  _CNPD2bits = 0x56
                    0x0058                  CNPD3 = 0x58
                    0x0058                  _CNPD3 = 0x58
                    0x0058                  _CNPD3bits = 0x58
                    0x005a                  CNPD4 = 0x5a
                    0x005a                  _CNPD4 = 0x5a
                    0x005a                  _CNPD4bits = 0x5a
                    0x005c                  CNPD5 = 0x5c
                    0x005c                  _CNPD5 = 0x5c
                    0x005c                  _CNPD5bits = 0x5c
                    0x005e                  CNPD6 = 0x5e
                    0x005e                  _CNPD6 = 0x5e
                    0x005e                  _CNPD6bits = 0x5e
                    0x0060                  CNEN1 = 0x60
                    0x0060                  _CNEN1 = 0x60
                    0x0060                  _CNEN1bits = 0x60
                    0x0062                  CNEN2 = 0x62
                    0x0062                  _CNEN2 = 0x62
                    0x0062                  _CNEN2bits = 0x62
                    0x0064                  CNEN3 = 0x64
                    0x0064                  _CNEN3 = 0x64
                    0x0064                  _CNEN3bits = 0x64
                    0x0066                  CNEN4 = 0x66
                    0x0066                  _CNEN4 = 0x66
                    0x0066                  _CNEN4bits = 0x66
                    0x0068                  CNEN5 = 0x68
                    0x0068                  _CNEN5 = 0x68
                    0x0068                  _CNEN5bits = 0x68
                    0x006a                  CNEN6 = 0x6a
                    0x006a                  _CNEN6 = 0x6a
                    0x006a                  _CNEN6bits = 0x6a
                    0x006c                  CNPU1 = 0x6c
                    0x006c                  _CNPU1 = 0x6c
                    0x006c                  _CNPU1bits = 0x6c
                    0x006e                  CNPU2 = 0x6e
                    0x006e                  _CNPU2 = 0x6e
                    0x006e                  _CNPU2bits = 0x6e
                    0x0070                  CNPU3 = 0x70
                    0x0070                  _CNPU3 = 0x70
                    0x0070                  _CNPU3bits = 0x70
                    0x0072                  CNPU4 = 0x72
                    0x0072                  _CNPU4 = 0x72
                    0x0072                  _CNPU4bits = 0x72
                    0x0074                  CNPU5 = 0x74
                    0x0074                  _CNPU5 = 0x74
                    0x0074                  _CNPU5bits = 0x74
                    0x0076                  CNPU6 = 0x76
                    0x0076                  _CNPU6 = 0x76
                    0x0076                  _CNPU6bits = 0x76
                    0x0080                  INTCON1 = 0x80
                    0x0080                  _INTCON1 = 0x80
                    0x0080                  _INTCON1bits = 0x80
                    0x0082                  INTCON2 = 0x82
                    0x0082                  _INTCON2 = 0x82
                    0x0082                  _INTCON2bits = 0x82
                    0x0084                  IFS0 = 0x84
                    0x0084                  _IFS0 = 0x84
                    0x0084                  _IFS0bits = 0x84
                    0x0086                  IFS1 = 0x86
                    0x0086                  _IFS1 = 0x86
                    0x0086                  _IFS1bits = 0x86
                    0x0088                  IFS2 = 0x88
                    0x0088                  _IFS2 = 0x88
                    0x0088                  _IFS2bits = 0x88
                    0x008a                  IFS3 = 0x8a
                    0x008a                  _IFS3 = 0x8a
                    0x008a                  _IFS3bits = 0x8a
                    0x008c                  IFS4 = 0x8c
                    0x008c                  _IFS4 = 0x8c
                    0x008c                  _IFS4bits = 0x8c
                    0x008e                  IFS5 = 0x8e
                    0x008e                  _IFS5 = 0x8e
                    0x008e                  _IFS5bits = 0x8e
                    0x0094                  IEC0 = 0x94
                    0x0094                  _IEC0 = 0x94
                    0x0094                  _IEC0bits = 0x94
                    0x0096                  IEC1 = 0x96
                    0x0096                  _IEC1 = 0x96
                    0x0096                  _IEC1bits = 0x96
                    0x0098                  IEC2 = 0x98
                    0x0098                  _IEC2 = 0x98
                    0x0098                  _IEC2bits = 0x98
                    0x009a                  IEC3 = 0x9a
                    0x009a                  _IEC3 = 0x9a
                    0x009a                  _IEC3bits = 0x9a
                    0x009c                  IEC4 = 0x9c
                    0x009c                  _IEC4 = 0x9c
                    0x009c                  _IEC4bits = 0x9c
                    0x009e                  IEC5 = 0x9e
                    0x009e                  _IEC5 = 0x9e
                    0x009e                  _IEC5bits = 0x9e
                    0x00a4                  IPC0 = 0xa4
                    0x00a4                  _IPC0 = 0xa4
                    0x00a4                  _IPC0bits = 0xa4
                    0x00a6                  IPC1 = 0xa6
                    0x00a6                  _IPC1 = 0xa6
                    0x00a6                  _IPC1bits = 0xa6
                    0x00a8                  IPC2 = 0xa8
                    0x00a8                  _IPC2 = 0xa8
                    0x00a8                  _IPC2bits = 0xa8
                    0x00aa                  IPC3 = 0xaa
                    0x00aa                  _IPC3 = 0xaa
                    0x00aa                  _IPC3bits = 0xaa
                    0x00ac                  IPC4 = 0xac
                    0x00ac                  _IPC4 = 0xac
                    0x00ac                  _IPC4bits = 0xac
                    0x00ae                  IPC5 = 0xae
                    0x00ae                  _IPC5 = 0xae
                    0x00ae                  _IPC5bits = 0xae
                    0x00b0                  IPC6 = 0xb0
                    0x00b0                  _IPC6 = 0xb0
                    0x00b0                  _IPC6bits = 0xb0
                    0x00b2                  IPC7 = 0xb2
                    0x00b2                  _IPC7 = 0xb2
                    0x00b2                  _IPC7bits = 0xb2
                    0x00b4                  IPC8 = 0xb4
                    0x00b4                  _IPC8 = 0xb4
                    0x00b4                  _IPC8bits = 0xb4
                    0x00b6                  IPC9 = 0xb6
                    0x00b6                  _IPC9 = 0xb6
                    0x00b6                  _IPC9bits = 0xb6
                    0x00b8                  IPC10 = 0xb8
                    0x00b8                  _IPC10 = 0xb8
                    0x00b8                  _IPC10bits = 0xb8
                    0x00ba                  IPC11 = 0xba
                    0x00ba                  _IPC11 = 0xba
                    0x00ba                  _IPC11bits = 0xba
                    0x00bc                  IPC12 = 0xbc
                    0x00bc                  _IPC12 = 0xbc
                    0x00bc                  _IPC12bits = 0xbc
                    0x00be                  IPC13 = 0xbe
                    0x00be                  _IPC13 = 0xbe
                    0x00be                  _IPC13bits = 0xbe
                    0x00c2                  IPC15 = 0xc2
                    0x00c2                  _IPC15 = 0xc2
                    0x00c2                  _IPC15bits = 0xc2
                    0x00c4                  IPC16 = 0xc4
                    0x00c4                  _IPC16 = 0xc4
                    0x00c4                  _IPC16bits = 0xc4
                    0x00c8                  IPC18 = 0xc8
                    0x00c8                  _IPC18 = 0xc8
                    0x00c8                  _IPC18bits = 0xc8
                    0x00ca                  IPC19 = 0xca
                    0x00ca                  _IPC19 = 0xca
                    0x00ca                  _IPC19bits = 0xca
                    0x00cc                  IPC20 = 0xcc
                    0x00cc                  _IPC20 = 0xcc
                    0x00cc                  _IPC20bits = 0xcc
                    0x00ce                  IPC21 = 0xce
                    0x00ce                  _IPC21 = 0xce
                    0x00ce                  _IPC21bits = 0xce
                    0x00d0                  IPC22 = 0xd0
                    0x00d0                  _IPC22 = 0xd0
                    0x00d0                  _IPC22bits = 0xd0
                    0x00d2                  IPC23 = 0xd2
                    0x00d2                  _IPC23 = 0xd2
                    0x00d2                  _IPC23bits = 0xd2
                    0x0100                  TMR1 = 0x100
                    0x0100                  _TMR1 = 0x100
                    0x0102                  PR1 = 0x102
                    0x0102                  _PR1 = 0x102
                    0x0104                  T1CON = 0x104
                    0x0104                  _T1CON = 0x104
                    0x0104                  _T1CONbits = 0x104
                    0x0106                  TMR2 = 0x106
                    0x0106                  _TMR2 = 0x106
                    0x0108                  TMR3HLD = 0x108
                    0x0108                  _TMR3HLD = 0x108
                    0x010a                  TMR3 = 0x10a
                    0x010a                  _TMR3 = 0x10a
                    0x010c                  PR2 = 0x10c
                    0x010c                  _PR2 = 0x10c
                    0x010e                  PR3 = 0x10e
                    0x010e                  _PR3 = 0x10e
                    0x0110                  T2CON = 0x110
                    0x0110                  _T2CON = 0x110
                    0x0110                  _T2CONbits = 0x110
                    0x0112                  T3CON = 0x112
                    0x0112                  _T3CON = 0x112
                    0x0112                  _T3CONbits = 0x112
                    0x0114                  TMR4 = 0x114
                    0x0114                  _TMR4 = 0x114
                    0x0116                  TMR5HLD = 0x116
                    0x0116                  _TMR5HLD = 0x116
                    0x0118                  TMR5 = 0x118
                    0x0118                  _TMR5 = 0x118
                    0x011a                  PR4 = 0x11a
                    0x011a                  _PR4 = 0x11a
                    0x011c                  PR5 = 0x11c
                    0x011c                  _PR5 = 0x11c
                    0x011e                  T4CON = 0x11e
                    0x011e                  _T4CON = 0x11e
                    0x011e                  _T4CONbits = 0x11e
                    0x0120                  T5CON = 0x120
                    0x0120                  _T5CON = 0x120
                    0x0120                  _T5CONbits = 0x120
                    0x0140                  IC1CON1 = 0x140
                    0x0140                  _IC1CON1 = 0x140
                    0x0140                  _IC1CON1bits = 0x140
                    0x0142                  IC1CON2 = 0x142
                    0x0142                  _IC1CON2 = 0x142
                    0x0142                  _IC1CON2bits = 0x142
                    0x0144                  IC1BUF = 0x144
                    0x0144                  _IC1BUF = 0x144
                    0x0146                  IC1TMR = 0x146
                    0x0146                  _IC1TMR = 0x146
                    0x0148                  IC2CON1 = 0x148
                    0x0148                  _IC2CON1 = 0x148
                    0x0148                  _IC2CON1bits = 0x148
                    0x014a                  IC2CON2 = 0x14a
                    0x014a                  _IC2CON2 = 0x14a
                    0x014a                  _IC2CON2bits = 0x14a
                    0x014c                  IC2BUF = 0x14c
                    0x014c                  _IC2BUF = 0x14c
                    0x014e                  IC2TMR = 0x14e
                    0x014e                  _IC2TMR = 0x14e
                    0x0150                  IC3CON1 = 0x150
                    0x0150                  _IC3CON1 = 0x150
                    0x0150                  _IC3CON1bits = 0x150
                    0x0152                  IC3CON2 = 0x152
                    0x0152                  _IC3CON2 = 0x152
                    0x0152                  _IC3CON2bits = 0x152
                    0x0154                  IC3BUF = 0x154
                    0x0154                  _IC3BUF = 0x154
                    0x0156                  IC3TMR = 0x156
                    0x0156                  _IC3TMR = 0x156
                    0x0158                  IC4CON1 = 0x158
                    0x0158                  _IC4CON1 = 0x158
                    0x0158                  _IC4CON1bits = 0x158
                    0x015a                  IC4CON2 = 0x15a
                    0x015a                  _IC4CON2 = 0x15a
                    0x015a                  _IC4CON2bits = 0x15a
                    0x015c                  IC4BUF = 0x15c
                    0x015c                  _IC4BUF = 0x15c
                    0x015e                  IC4TMR = 0x15e
                    0x015e                  _IC4TMR = 0x15e
                    0x0160                  IC5CON1 = 0x160
                    0x0160                  _IC5CON1 = 0x160
                    0x0160                  _IC5CON1bits = 0x160
                    0x0162                  IC5CON2 = 0x162
                    0x0162                  _IC5CON2 = 0x162
                    0x0162                  _IC5CON2bits = 0x162
                    0x0164                  IC5BUF = 0x164
                    0x0164                  _IC5BUF = 0x164
                    0x0166                  IC5TMR = 0x166
                    0x0166                  _IC5TMR = 0x166
                    0x0168                  IC6CON1 = 0x168
                    0x0168                  _IC6CON1 = 0x168
                    0x0168                  _IC6CON1bits = 0x168
                    0x016a                  IC6CON2 = 0x16a
                    0x016a                  _IC6CON2 = 0x16a
                    0x016a                  _IC6CON2bits = 0x16a
                    0x016c                  IC6BUF = 0x16c
                    0x016c                  _IC6BUF = 0x16c
                    0x016e                  IC6TMR = 0x16e
                    0x016e                  _IC6TMR = 0x16e
                    0x0170                  IC7CON1 = 0x170
                    0x0170                  _IC7CON1 = 0x170
                    0x0170                  _IC7CON1bits = 0x170
                    0x0172                  IC7CON2 = 0x172
                    0x0172                  _IC7CON2 = 0x172
                    0x0172                  _IC7CON2bits = 0x172
                    0x0174                  IC7BUF = 0x174
                    0x0174                  _IC7BUF = 0x174
                    0x0176                  IC7TMR = 0x176
                    0x0176                  _IC7TMR = 0x176
                    0x0178                  IC8CON1 = 0x178
                    0x0178                  _IC8CON1 = 0x178
                    0x0178                  _IC8CON1bits = 0x178
                    0x017a                  IC8CON2 = 0x17a
                    0x017a                  _IC8CON2 = 0x17a
                    0x017a                  _IC8CON2bits = 0x17a
                    0x017c                  IC8BUF = 0x17c
                    0x017c                  _IC8BUF = 0x17c
                    0x017e                  IC8TMR = 0x17e
                    0x017e                  _IC8TMR = 0x17e
                    0x0180                  IC9CON1 = 0x180
                    0x0180                  _IC9CON1 = 0x180
                    0x0180                  _IC9CON1bits = 0x180
                    0x0182                  IC9CON2 = 0x182
                    0x0182                  _IC9CON2 = 0x182
                    0x0182                  _IC9CON2bits = 0x182
                    0x0184                  IC9BUF = 0x184
                    0x0184                  _IC9BUF = 0x184
                    0x0186                  IC9TMR = 0x186
                    0x0186                  _IC9TMR = 0x186
                    0x0190                  OC1CON1 = 0x190
                    0x0190                  _OC1CON1 = 0x190
                    0x0190                  _OC1CON1bits = 0x190
                    0x0192                  OC1CON2 = 0x192
                    0x0192                  _OC1CON2 = 0x192
                    0x0192                  _OC1CON2bits = 0x192
                    0x0194                  OC1RS = 0x194
                    0x0194                  _OC1RS = 0x194
                    0x0196                  OC1R = 0x196
                    0x0196                  _OC1R = 0x196
                    0x0198                  OC1TMR = 0x198
                    0x0198                  _OC1TMR = 0x198
                    0x019a                  OC2CON1 = 0x19a
                    0x019a                  _OC2CON1 = 0x19a
                    0x019a                  _OC2CON1bits = 0x19a
                    0x019c                  OC2CON2 = 0x19c
                    0x019c                  _OC2CON2 = 0x19c
                    0x019c                  _OC2CON2bits = 0x19c
                    0x019e                  OC2RS = 0x19e
                    0x019e                  _OC2RS = 0x19e
                    0x01a0                  OC2R = 0x1a0
                    0x01a0                  _OC2R = 0x1a0
                    0x01a2                  OC2TMR = 0x1a2
                    0x01a2                  _OC2TMR = 0x1a2
                    0x01a4                  OC3CON1 = 0x1a4
                    0x01a4                  _OC3CON1 = 0x1a4
                    0x01a4                  _OC3CON1bits = 0x1a4
                    0x01a6                  OC3CON2 = 0x1a6
                    0x01a6                  _OC3CON2 = 0x1a6
                    0x01a6                  _OC3CON2bits = 0x1a6
                    0x01a8                  OC3RS = 0x1a8
                    0x01a8                  _OC3RS = 0x1a8
                    0x01aa                  OC3R = 0x1aa
                    0x01aa                  _OC3R = 0x1aa
                    0x01ac                  OC3TMR = 0x1ac
                    0x01ac                  _OC3TMR = 0x1ac
                    0x01ae                  OC4CON1 = 0x1ae
                    0x01ae                  _OC4CON1 = 0x1ae
                    0x01ae                  _OC4CON1bits = 0x1ae
                    0x01b0                  OC4CON2 = 0x1b0
                    0x01b0                  _OC4CON2 = 0x1b0
                    0x01b0                  _OC4CON2bits = 0x1b0
                    0x01b2                  OC4RS = 0x1b2
                    0x01b2                  _OC4RS = 0x1b2
                    0x01b4                  OC4R = 0x1b4
                    0x01b4                  _OC4R = 0x1b4
                    0x01b6                  OC4TMR = 0x1b6
                    0x01b6                  _OC4TMR = 0x1b6
                    0x01b8                  OC5CON1 = 0x1b8
                    0x01b8                  _OC5CON1 = 0x1b8
                    0x01b8                  _OC5CON1bits = 0x1b8
                    0x01ba                  OC5CON2 = 0x1ba
                    0x01ba                  _OC5CON2 = 0x1ba
                    0x01ba                  _OC5CON2bits = 0x1ba
                    0x01bc                  OC5RS = 0x1bc
                    0x01bc                  _OC5RS = 0x1bc
                    0x01be                  OC5R = 0x1be
                    0x01be                  _OC5R = 0x1be
                    0x01c0                  OC5TMR = 0x1c0
                    0x01c0                  _OC5TMR = 0x1c0
                    0x01c2                  OC6CON1 = 0x1c2
                    0x01c2                  _OC6CON1 = 0x1c2
                    0x01c2                  _OC6CON1bits = 0x1c2
                    0x01c4                  OC6CON2 = 0x1c4
                    0x01c4                  _OC6CON2 = 0x1c4
                    0x01c4                  _OC6CON2bits = 0x1c4
                    0x01c6                  OC6RS = 0x1c6
                    0x01c6                  _OC6RS = 0x1c6
                    0x01c8                  OC6R = 0x1c8
                    0x01c8                  _OC6R = 0x1c8
                    0x01ca                  OC6TMR = 0x1ca
                    0x01ca                  _OC6TMR = 0x1ca
                    0x01cc                  OC7CON1 = 0x1cc
                    0x01cc                  _OC7CON1 = 0x1cc
                    0x01cc                  _OC7CON1bits = 0x1cc
                    0x01ce                  OC7CON2 = 0x1ce
                    0x01ce                  _OC7CON2 = 0x1ce
                    0x01ce                  _OC7CON2bits = 0x1ce
                    0x01d0                  OC7RS = 0x1d0
                    0x01d0                  _OC7RS = 0x1d0
                    0x01d2                  OC7R = 0x1d2
                    0x01d2                  _OC7R = 0x1d2
                    0x01d4                  OC7TMR = 0x1d4
                    0x01d4                  _OC7TMR = 0x1d4
                    0x01d6                  OC8CON1 = 0x1d6
                    0x01d6                  _OC8CON1 = 0x1d6
                    0x01d6                  _OC8CON1bits = 0x1d6
                    0x01d8                  OC8CON2 = 0x1d8
                    0x01d8                  _OC8CON2 = 0x1d8
                    0x01d8                  _OC8CON2bits = 0x1d8
                    0x01da                  OC8RS = 0x1da
                    0x01da                  _OC8RS = 0x1da
                    0x01dc                  OC8R = 0x1dc
                    0x01dc                  _OC8R = 0x1dc
                    0x01de                  OC8TMR = 0x1de
                    0x01de                  _OC8TMR = 0x1de
                    0x01e0                  OC9CON1 = 0x1e0
                    0x01e0                  _OC9CON1 = 0x1e0
                    0x01e0                  _OC9CON1bits = 0x1e0
                    0x01e2                  OC9CON2 = 0x1e2
                    0x01e2                  _OC9CON2 = 0x1e2
                    0x01e2                  _OC9CON2bits = 0x1e2
                    0x01e4                  OC9RS = 0x1e4
                    0x01e4                  _OC9RS = 0x1e4
                    0x01e6                  OC9R = 0x1e6
                    0x01e6                  _OC9R = 0x1e6
                    0x01e8                  OC9TMR = 0x1e8
                    0x01e8                  _OC9TMR = 0x1e8
                    0x0200                  I2C1RCV = 0x200
                    0x0200                  _I2C1RCV = 0x200
                    0x0202                  I2C1TRN = 0x202
                    0x0202                  _I2C1TRN = 0x202
                    0x0204                  I2C1BRG = 0x204
                    0x0204                  _I2C1BRG = 0x204
                    0x0206                  I2C1CON = 0x206
                    0x0206                  _I2C1CON = 0x206
                    0x0206                  _I2C1CONbits = 0x206
                    0x0208                  I2C1STAT = 0x208
                    0x0208                  _I2C1STAT = 0x208
                    0x0208                  _I2C1STATbits = 0x208
                    0x020a                  I2C1ADD = 0x20a
                    0x020a                  _I2C1ADD = 0x20a
                    0x020c                  I2C1MSK = 0x20c
                    0x020c                  _I2C1MSK = 0x20c
                    0x0210                  I2C2RCV = 0x210
                    0x0210                  _I2C2RCV = 0x210
                    0x0212                  I2C2TRN = 0x212
                    0x0212                  _I2C2TRN = 0x212
                    0x0214                  I2C2BRG = 0x214
                    0x0214                  _I2C2BRG = 0x214
                    0x0216                  I2C2CON = 0x216
                    0x0216                  _I2C2CON = 0x216
                    0x0216                  _I2C2CONbits = 0x216
                    0x0218                  I2C2STAT = 0x218
                    0x0218                  _I2C2STAT = 0x218
                    0x0218                  _I2C2STATbits = 0x218
                    0x021a                  I2C2ADD = 0x21a
                    0x021a                  _I2C2ADD = 0x21a
                    0x021c                  I2C2MSK = 0x21c
                    0x021c                  _I2C2MSK = 0x21c
                    0x0220                  U1MODE = 0x220
                    0x0220                  _U1MODE = 0x220
                    0x0220                  _U1MODEbits = 0x220
                    0x0222                  U1STA = 0x222
                    0x0222                  _U1STA = 0x222
                    0x0222                  _U1STAbits = 0x222
                    0x0224                  U1TXREG = 0x224
                    0x0224                  _U1TXREG = 0x224
                    0x0226                  U1RXREG = 0x226
                    0x0226                  _U1RXREG = 0x226
                    0x0228                  U1BRG = 0x228
                    0x0228                  _U1BRG = 0x228
                    0x0230                  U2MODE = 0x230
                    0x0230                  _U2MODE = 0x230
                    0x0230                  _U2MODEbits = 0x230
                    0x0232                  U2STA = 0x232
                    0x0232                  _U2STA = 0x232
                    0x0232                  _U2STAbits = 0x232
                    0x0234                  U2TXREG = 0x234
                    0x0234                  _U2TXREG = 0x234
                    0x0236                  U2RXREG = 0x236
                    0x0236                  _U2RXREG = 0x236
                    0x0238                  U2BRG = 0x238
                    0x0238                  _U2BRG = 0x238
                    0x0240                  SPI1STAT = 0x240
                    0x0240                  _SPI1STAT = 0x240
                    0x0240                  _SPI1STATbits = 0x240
                    0x0242                  SPI1CON1 = 0x242
                    0x0242                  _SPI1CON1 = 0x242
                    0x0242                  _SPI1CON1bits = 0x242
                    0x0244                  SPI1CON2 = 0x244
                    0x0244                  _SPI1CON2 = 0x244
                    0x0244                  _SPI1CON2bits = 0x244
                    0x0248                  SPI1BUF = 0x248
                    0x0248                  _SPI1BUF = 0x248
                    0x0250                  U3MODE = 0x250
                    0x0250                  _U3MODE = 0x250
                    0x0250                  _U3MODEbits = 0x250
                    0x0252                  U3STA = 0x252
                    0x0252                  _U3STA = 0x252
                    0x0252                  _U3STAbits = 0x252
                    0x0254                  U3TXREG = 0x254
                    0x0254                  _U3TXREG = 0x254
                    0x0256                  U3RXREG = 0x256
                    0x0256                  _U3RXREG = 0x256
                    0x0258                  U3BRG = 0x258
                    0x0258                  _U3BRG = 0x258
                    0x0260                  SPI2STAT = 0x260
                    0x0260                  _SPI2STAT = 0x260
                    0x0260                  _SPI2STATbits = 0x260
                    0x0262                  SPI2CON1 = 0x262
                    0x0262                  _SPI2CON1 = 0x262
                    0x0262                  _SPI2CON1bits = 0x262
                    0x0264                  SPI2CON2 = 0x264
                    0x0264                  _SPI2CON2 = 0x264
                    0x0264                  _SPI2CON2bits = 0x264
                    0x0268                  SPI2BUF = 0x268
                    0x0268                  _SPI2BUF = 0x268
                    0x0270                  I2C3RCV = 0x270
                    0x0270                  _I2C3RCV = 0x270
                    0x0272                  I2C3TRN = 0x272
                    0x0272                  _I2C3TRN = 0x272
                    0x0274                  I2C3BRG = 0x274
                    0x0274                  _I2C3BRG = 0x274
                    0x0276                  I2C3CON = 0x276
                    0x0276                  _I2C3CON = 0x276
                    0x0276                  _I2C3CONbits = 0x276
                    0x0278                  I2C3STAT = 0x278
                    0x0278                  _I2C3STAT = 0x278
                    0x0278                  _I2C3STATbits = 0x278
                    0x027a                  I2C3ADD = 0x27a
                    0x027a                  _I2C3ADD = 0x27a
                    0x027c                  I2C3MSK = 0x27c
                    0x027c                  _I2C3MSK = 0x27c
                    0x0280                  SPI3STAT = 0x280
                    0x0280                  _SPI3STAT = 0x280
                    0x0280                  _SPI3STATbits = 0x280
                    0x0282                  SPI3CON1 = 0x282
                    0x0282                  _SPI3CON1 = 0x282
                    0x0282                  _SPI3CON1bits = 0x282
                    0x0284                  SPI3CON2 = 0x284
                    0x0284                  _SPI3CON2 = 0x284
                    0x0284                  _SPI3CON2bits = 0x284
                    0x0288                  SPI3BUF = 0x288
                    0x0288                  _SPI3BUF = 0x288
                    0x02b0                  U4MODE = 0x2b0
                    0x02b0                  _U4MODE = 0x2b0
                    0x02b0                  _U4MODEbits = 0x2b0
                    0x02b2                  U4STA = 0x2b2
                    0x02b2                  _U4STA = 0x2b2
                    0x02b2                  _U4STAbits = 0x2b2
                    0x02b4                  U4TXREG = 0x2b4
                    0x02b4                  _U4TXREG = 0x2b4
                    0x02b6                  U4RXREG = 0x2b6
                    0x02b6                  _U4RXREG = 0x2b6
                    0x02b8                  U4BRG = 0x2b8
                    0x02b8                  _U4BRG = 0x2b8
                    0x02c0                  TRISA = 0x2c0
                    0x02c0                  _TRISA = 0x2c0
                    0x02c0                  _TRISAbits = 0x2c0
                    0x02c2                  PORTA = 0x2c2
                    0x02c2                  _PORTA = 0x2c2
                    0x02c2                  _PORTAbits = 0x2c2
                    0x02c4                  LATA = 0x2c4
                    0x02c4                  _LATA = 0x2c4
                    0x02c4                  _LATAbits = 0x2c4
                    0x02c6                  ODCA = 0x2c6
                    0x02c6                  _ODCA = 0x2c6
                    0x02c6                  _ODCAbits = 0x2c6
                    0x02c8                  TRISB = 0x2c8
                    0x02c8                  _TRISB = 0x2c8
                    0x02c8                  _TRISBbits = 0x2c8
                    0x02ca                  PORTB = 0x2ca
                    0x02ca                  _PORTB = 0x2ca
                    0x02ca                  _PORTBbits = 0x2ca
                    0x02cc                  LATB = 0x2cc
                    0x02cc                  _LATB = 0x2cc
                    0x02cc                  _LATBbits = 0x2cc
                    0x02ce                  ODCB = 0x2ce
                    0x02ce                  _ODCB = 0x2ce
                    0x02ce                  _ODCBbits = 0x2ce
                    0x02d0                  TRISC = 0x2d0
                    0x02d0                  _TRISC = 0x2d0
                    0x02d0                  _TRISCbits = 0x2d0
                    0x02d2                  PORTC = 0x2d2
                    0x02d2                  _PORTC = 0x2d2
                    0x02d2                  _PORTCbits = 0x2d2
                    0x02d4                  LATC = 0x2d4
                    0x02d4                  _LATC = 0x2d4
                    0x02d4                  _LATCbits = 0x2d4
                    0x02d6                  ODCC = 0x2d6
                    0x02d6                  _ODCC = 0x2d6
                    0x02d6                  _ODCCbits = 0x2d6
                    0x02d8                  TRISD = 0x2d8
                    0x02d8                  _TRISD = 0x2d8
                    0x02d8                  _TRISDbits = 0x2d8
                    0x02da                  PORTD = 0x2da
                    0x02da                  _PORTD = 0x2da
                    0x02da                  _PORTDbits = 0x2da
                    0x02dc                  LATD = 0x2dc
                    0x02dc                  _LATD = 0x2dc
                    0x02dc                  _LATDbits = 0x2dc
                    0x02de                  ODCD = 0x2de
                    0x02de                  _ODCD = 0x2de
                    0x02de                  _ODCDbits = 0x2de
                    0x02e0                  TRISE = 0x2e0
                    0x02e0                  _TRISE = 0x2e0
                    0x02e0                  _TRISEbits = 0x2e0
                    0x02e2                  PORTE = 0x2e2
                    0x02e2                  _PORTE = 0x2e2
                    0x02e2                  _PORTEbits = 0x2e2
                    0x02e4                  LATE = 0x2e4
                    0x02e4                  _LATE = 0x2e4
                    0x02e4                  _LATEbits = 0x2e4
                    0x02e6                  ODCE = 0x2e6
                    0x02e6                  _ODCE = 0x2e6
                    0x02e6                  _ODCEbits = 0x2e6
                    0x02e8                  TRISF = 0x2e8
                    0x02e8                  _TRISF = 0x2e8
                    0x02e8                  _TRISFbits = 0x2e8
                    0x02ea                  PORTF = 0x2ea
                    0x02ea                  _PORTF = 0x2ea
                    0x02ea                  _PORTFbits = 0x2ea
                    0x02ec                  LATF = 0x2ec
                    0x02ec                  _LATF = 0x2ec
                    0x02ec                  _LATFbits = 0x2ec
                    0x02ee                  ODCF = 0x2ee
                    0x02ee                  _ODCF = 0x2ee
                    0x02ee                  _ODCFbits = 0x2ee
                    0x02f0                  TRISG = 0x2f0
                    0x02f0                  _TRISG = 0x2f0
                    0x02f0                  _TRISGbits = 0x2f0
                    0x02f2                  PORTG = 0x2f2
                    0x02f2                  _PORTG = 0x2f2
                    0x02f2                  _PORTGbits = 0x2f2
                    0x02f4                  LATG = 0x2f4
                    0x02f4                  _LATG = 0x2f4
                    0x02f4                  _LATGbits = 0x2f4
                    0x02f6                  ODCG = 0x2f6
                    0x02f6                  _ODCG = 0x2f6
                    0x02f6                  _ODCGbits = 0x2f6
                    0x02fc                  PADCFG1 = 0x2fc
                    0x02fc                  _PADCFG1 = 0x2fc
                    0x02fc                  _PADCFG1bits = 0x2fc
                    0x0300                  ADC1BUF0 = 0x300
                    0x0300                  _ADC1BUF0 = 0x300
                    0x0302                  ADC1BUF1 = 0x302
                    0x0302                  _ADC1BUF1 = 0x302
                    0x0304                  ADC1BUF2 = 0x304
                    0x0304                  _ADC1BUF2 = 0x304
                    0x0306                  ADC1BUF3 = 0x306
                    0x0306                  _ADC1BUF3 = 0x306
                    0x0308                  ADC1BUF4 = 0x308
                    0x0308                  _ADC1BUF4 = 0x308
                    0x030a                  ADC1BUF5 = 0x30a
                    0x030a                  _ADC1BUF5 = 0x30a
                    0x030c                  ADC1BUF6 = 0x30c
                    0x030c                  _ADC1BUF6 = 0x30c
                    0x030e                  ADC1BUF7 = 0x30e
                    0x030e                  _ADC1BUF7 = 0x30e
                    0x0310                  ADC1BUF8 = 0x310
                    0x0310                  _ADC1BUF8 = 0x310
                    0x0312                  ADC1BUF9 = 0x312
                    0x0312                  _ADC1BUF9 = 0x312
                    0x0314                  ADC1BUFA = 0x314
                    0x0314                  _ADC1BUFA = 0x314
                    0x0316                  ADC1BUFB = 0x316
                    0x0316                  _ADC1BUFB = 0x316
                    0x0318                  ADC1BUFC = 0x318
                    0x0318                  _ADC1BUFC = 0x318
                    0x031a                  ADC1BUFD = 0x31a
                    0x031a                  _ADC1BUFD = 0x31a
                    0x031c                  ADC1BUFE = 0x31c
                    0x031c                  _ADC1BUFE = 0x31c
                    0x031e                  ADC1BUFF = 0x31e
                    0x031e                  _ADC1BUFF = 0x31e
                    0x0320                  AD1CON1 = 0x320
                    0x0320                  _AD1CON1 = 0x320
                    0x0320                  _AD1CON1bits = 0x320
                    0x0322                  AD1CON2 = 0x322
                    0x0322                  _AD1CON2 = 0x322
                    0x0322                  _AD1CON2bits = 0x322
                    0x0324                  AD1CON3 = 0x324
                    0x0324                  _AD1CON3 = 0x324
                    0x0324                  _AD1CON3bits = 0x324
                    0x0328                  AD1CHS = 0x328
                    0x0328                  _AD1CHS = 0x328
                    0x0328                  _AD1CHSbits = 0x328
                    0x0328                  AD1CHS0 = 0x328
                    0x0328                  _AD1CHS0 = 0x328
                    0x0328                  _AD1CHS0bits = 0x328
                    0x032a                  AD1PCFGH = 0x32a
                    0x032a                  _AD1PCFGH = 0x32a
                    0x032a                  _AD1PCFGHbits = 0x32a
                    0x032c                  AD1PCFG = 0x32c
                    0x032c                  _AD1PCFG = 0x32c
                    0x032c                  _AD1PCFGbits = 0x32c
                    0x032c                  AD1PCFGL = 0x32c
                    0x032c                  _AD1PCFGL = 0x32c
                    0x032c                  _AD1PCFGLbits = 0x32c
                    0x0330                  AD1CSSL = 0x330
                    0x0330                  _AD1CSSL = 0x330
                    0x0330                  _AD1CSSLbits = 0x330
                    0x0332                  AD1CSSH = 0x332
                    0x0332                  _AD1CSSH = 0x332
                    0x0332                  _AD1CSSHbits = 0x332
                    0x033c                  CTMUCON = 0x33c
                    0x033c                  _CTMUCON = 0x33c
                    0x033c                  _CTMUCONbits = 0x33c
                    0x033e                  CTMUICON = 0x33e
                    0x033e                  _CTMUICON = 0x33e
                    0x033e                  _CTMUICONbits = 0x33e
                    0x0600                  PMCON = 0x600
                    0x0600                  _PMCON = 0x600
                    0x0600                  _PMCONbits = 0x600
                    0x0602                  PMMODE = 0x602
                    0x0602                  _PMMODE = 0x602
                    0x0602                  _PMMODEbits = 0x602
                    0x0604                  PMADDR = 0x604
                    0x0604                  _PMADDR = 0x604
                    0x0604                  _PMADDRbits = 0x604
                    0x0604                  PMDOUT1 = 0x604
                    0x0604                  _PMDOUT1 = 0x604
                    0x0604                  _PMDOUT1bits = 0x604
                    0x0606                  PMDOUT2 = 0x606
                    0x0606                  _PMDOUT2 = 0x606
                    0x0608                  PMDIN1 = 0x608
                    0x0608                  _PMDIN1 = 0x608
                    0x060a                  PMDIN2 = 0x60a
                    0x060a                  _PMDIN2 = 0x60a
                    0x060c                  PMAEN = 0x60c
                    0x060c                  _PMAEN = 0x60c
                    0x060c                  _PMAENbits = 0x60c
                    0x060e                  PMSTAT = 0x60e
                    0x060e                  _PMSTAT = 0x60e
                    0x060e                  _PMSTATbits = 0x60e
                    0x0620                  ALRMVAL = 0x620
                    0x0620                  _ALRMVAL = 0x620
                    0x0622                  ALCFGRPT = 0x622
                    0x0622                  _ALCFGRPT = 0x622
                    0x0622                  _ALCFGRPTbits = 0x622
                    0x0624                  RTCVAL = 0x624
                    0x0624                  _RTCVAL = 0x624
                    0x0626                  RCFGCAL = 0x626
                    0x0626                  _RCFGCAL = 0x626
                    0x0626                  _RCFGCALbits = 0x626
                    0x0630                  CMSTAT = 0x630
                    0x0630                  _CMSTAT = 0x630
                    0x0630                  _CMSTATbits = 0x630
                    0x0632                  CVRCON = 0x632
                    0x0632                  _CVRCON = 0x632
                    0x0632                  _CVRCONbits = 0x632
                    0x0634                  CM1CON = 0x634
                    0x0634                  _CM1CON = 0x634
                    0x0634                  _CM1CONbits = 0x634
                    0x0636                  CM2CON = 0x636
                    0x0636                  _CM2CON = 0x636
                    0x0636                  _CM2CONbits = 0x636
                    0x0638                  CM3CON = 0x638
                    0x0638                  _CM3CON = 0x638
                    0x0638                  _CM3CONbits = 0x638
                    0x0640                  CRCCON = 0x640
                    0x0640                  _CRCCON = 0x640
                    0x0640                  _CRCCONbits = 0x640
                    0x0642                  CRCXOR = 0x642
                    0x0642                  _CRCXOR = 0x642
                    0x0642                  _CRCXORbits = 0x642
                    0x0644                  CRCDAT = 0x644
                    0x0644                  _CRCDAT = 0x644
                    0x0646                  CRCWDAT = 0x646
                    0x0646                  _CRCWDAT = 0x646
                    0x0680                  RPINR0 = 0x680
                    0x0680                  _RPINR0 = 0x680
                    0x0680                  _RPINR0bits = 0x680
                    0x0682                  RPINR1 = 0x682
                    0x0682                  _RPINR1 = 0x682
                    0x0682                  _RPINR1bits = 0x682
                    0x0684                  RPINR2 = 0x684
                    0x0684                  _RPINR2 = 0x684
                    0x0684                  _RPINR2bits = 0x684
                    0x0686                  RPINR3 = 0x686
                    0x0686                  _RPINR3 = 0x686
                    0x0686                  _RPINR3bits = 0x686
                    0x0688                  RPINR4 = 0x688
                    0x0688                  _RPINR4 = 0x688
                    0x0688                  _RPINR4bits = 0x688
                    0x068e                  RPINR7 = 0x68e
                    0x068e                  _RPINR7 = 0x68e
                    0x068e                  _RPINR7bits = 0x68e
                    0x0690                  RPINR8 = 0x690
                    0x0690                  _RPINR8 = 0x690
                    0x0690                  _RPINR8bits = 0x690
                    0x0692                  RPINR9 = 0x692
                    0x0692                  _RPINR9 = 0x692
                    0x0692                  _RPINR9bits = 0x692
                    0x0694                  RPINR10 = 0x694
                    0x0694                  _RPINR10 = 0x694
                    0x0694                  _RPINR10bits = 0x694
                    0x0696                  RPINR11 = 0x696
                    0x0696                  _RPINR11 = 0x696
                    0x0696                  _RPINR11bits = 0x696
                    0x069e                  RPINR15 = 0x69e
                    0x069e                  _RPINR15 = 0x69e
                    0x069e                  _RPINR15bits = 0x69e
                    0x06a2                  RPINR17 = 0x6a2
                    0x06a2                  _RPINR17 = 0x6a2
                    0x06a2                  _RPINR17bits = 0x6a2
                    0x06a4                  RPINR18 = 0x6a4
                    0x06a4                  _RPINR18 = 0x6a4
                    0x06a4                  _RPINR18bits = 0x6a4
                    0x06a6                  RPINR19 = 0x6a6
                    0x06a6                  _RPINR19 = 0x6a6
                    0x06a6                  _RPINR19bits = 0x6a6
                    0x06a8                  RPINR20 = 0x6a8
                    0x06a8                  _RPINR20 = 0x6a8
                    0x06a8                  _RPINR20bits = 0x6a8
                    0x06aa                  RPINR21 = 0x6aa
                    0x06aa                  _RPINR21 = 0x6aa
                    0x06aa                  _RPINR21bits = 0x6aa
                    0x06ac                  RPINR22 = 0x6ac
                    0x06ac                  _RPINR22 = 0x6ac
                    0x06ac                  _RPINR22bits = 0x6ac
                    0x06ae                  RPINR23 = 0x6ae
                    0x06ae                  _RPINR23 = 0x6ae
                    0x06ae                  _RPINR23bits = 0x6ae
                    0x06b6                  RPINR27 = 0x6b6
                    0x06b6                  _RPINR27 = 0x6b6
                    0x06b6                  _RPINR27bits = 0x6b6
                    0x06b8                  RPINR28 = 0x6b8
                    0x06b8                  _RPINR28 = 0x6b8
                    0x06b8                  _RPINR28bits = 0x6b8
                    0x06ba                  RPINR29 = 0x6ba
                    0x06ba                  _RPINR29 = 0x6ba
                    0x06ba                  _RPINR29bits = 0x6ba
                    0x06c0                  RPOR0 = 0x6c0
                    0x06c0                  _RPOR0 = 0x6c0
                    0x06c0                  _RPOR0bits = 0x6c0
                    0x06c2                  RPOR1 = 0x6c2
                    0x06c2                  _RPOR1 = 0x6c2
                    0x06c2                  _RPOR1bits = 0x6c2
                    0x06c4                  RPOR2 = 0x6c4
                    0x06c4                  _RPOR2 = 0x6c4
                    0x06c4                  _RPOR2bits = 0x6c4
                    0x06c6                  RPOR3 = 0x6c6
                    0x06c6                  _RPOR3 = 0x6c6
                    0x06c6                  _RPOR3bits = 0x6c6
                    0x06c8                  RPOR4 = 0x6c8
                    0x06c8                  _RPOR4 = 0x6c8
                    0x06c8                  _RPOR4bits = 0x6c8
                    0x06ca                  RPOR5 = 0x6ca
                    0x06ca                  _RPOR5 = 0x6ca
                    0x06ca                  _RPOR5bits = 0x6ca
                    0x06cc                  RPOR6 = 0x6cc
                    0x06cc                  _RPOR6 = 0x6cc
                    0x06cc                  _RPOR6bits = 0x6cc
                    0x06ce                  RPOR7 = 0x6ce
                    0x06ce                  _RPOR7 = 0x6ce
                    0x06ce                  _RPOR7bits = 0x6ce
                    0x06d0                  RPOR8 = 0x6d0
                    0x06d0                  _RPOR8 = 0x6d0
                    0x06d0                  _RPOR8bits = 0x6d0
                    0x06d2                  RPOR9 = 0x6d2
                    0x06d2                  _RPOR9 = 0x6d2
                    0x06d2                  _RPOR9bits = 0x6d2
                    0x06d4                  RPOR10 = 0x6d4
                    0x06d4                  _RPOR10 = 0x6d4
                    0x06d4                  _RPOR10bits = 0x6d4
                    0x06d6                  RPOR11 = 0x6d6
                    0x06d6                  _RPOR11 = 0x6d6
                    0x06d6                  _RPOR11bits = 0x6d6
                    0x06d8                  RPOR12 = 0x6d8
                    0x06d8                  _RPOR12 = 0x6d8
                    0x06d8                  _RPOR12bits = 0x6d8
                    0x06da                  RPOR13 = 0x6da
                    0x06da                  _RPOR13 = 0x6da
                    0x06da                  _RPOR13bits = 0x6da
                    0x06dc                  RPOR14 = 0x6dc
                    0x06dc                  _RPOR14 = 0x6dc
                    0x06dc                  _RPOR14bits = 0x6dc
                    0x06de                  RPOR15 = 0x6de
                    0x06de                  _RPOR15 = 0x6de
                    0x06de                  _RPOR15bits = 0x6de
                    0x0740                  RCON = 0x740
                    0x0740                  _RCON = 0x740
                    0x0740                  _RCONbits = 0x740
                    0x0742                  OSCCON = 0x742
                    0x0742                  _OSCCON = 0x742
                    0x0742                  _OSCCONbits = 0x742
                    0x0742                  OSCCONL = 0x742
                    0x0742                  _OSCCONL = 0x742
                    0x0743                  OSCCONH = 0x743
                    0x0743                  _OSCCONH = 0x743
                    0x0744                  CLKDIV = 0x744
                    0x0744                  _CLKDIV = 0x744
                    0x0744                  _CLKDIVbits = 0x744
                    0x0748                  OSCTUN = 0x748
                    0x0748                  _OSCTUN = 0x748
                    0x0748                  _OSCTUNbits = 0x748
                    0x074e                  REFOCON = 0x74e
                    0x074e                  _REFOCON = 0x74e
                    0x074e                  _REFOCONbits = 0x74e
                    0x0760                  NVMCON = 0x760
                    0x0760                  _NVMCON = 0x760
                    0x0760                  _NVMCONbits = 0x760
                    0x0766                  NVMKEY = 0x766
                    0x0766                  _NVMKEY = 0x766
                    0x0770                  PMD1 = 0x770
                    0x0770                  _PMD1 = 0x770
                    0x0770                  _PMD1bits = 0x770
                    0x0772                  PMD2 = 0x772
                    0x0772                  _PMD2 = 0x772
                    0x0772                  _PMD2bits = 0x772
                    0x0774                  PMD3 = 0x774
                    0x0774                  _PMD3 = 0x774
                    0x0774                  _PMD3bits = 0x774
                    0x0776                  PMD4 = 0x776
                    0x0776                  _PMD4 = 0x776
                    0x0776                  _PMD4bits = 0x776
                    0x0778                  PMD5 = 0x778
                    0x0778                  _PMD5 = 0x778
                    0x0778                  _PMD5bits = 0x778
                    0x077a                  PMD6 = 0x77a
                    0x077a                  _PMD6 = 0x77a
                    0x077a                  _PMD6bits = 0x77a
                    0x0144                  IC1 = 0x144
                    0x0144                  _IC1 = 0x144
                    0x014c                  IC2 = 0x14c
                    0x014c                  _IC2 = 0x14c
                    0x0154                  IC3 = 0x154
                    0x0154                  _IC3 = 0x154
                    0x015c                  IC4 = 0x15c
                    0x015c                  _IC4 = 0x15c
                    0x0164                  IC5 = 0x164
                    0x0164                  _IC5 = 0x164
                    0x016c                  IC6 = 0x16c
                    0x016c                  _IC6 = 0x16c
                    0x0174                  IC7 = 0x174
                    0x0174                  _IC7 = 0x174
                    0x017c                  IC8 = 0x17c
                    0x017c                  _IC8 = 0x17c
                    0x0194                  OC1 = 0x194
                    0x0194                  _OC1 = 0x194
                    0x019e                  OC2 = 0x19e
                    0x019e                  _OC2 = 0x19e
                    0x01a8                  OC3 = 0x1a8
                    0x01a8                  _OC3 = 0x1a8
                    0x01b2                  OC4 = 0x1b2
                    0x01b2                  _OC4 = 0x1b2
                    0x01bc                  OC5 = 0x1bc
                    0x01bc                  _OC5 = 0x1bc
                    0x01c6                  OC6 = 0x1c6
                    0x01c6                  _OC6 = 0x1c6
                    0x01d0                  OC7 = 0x1d0
                    0x01d0                  _OC7 = 0x1d0
                    0x01da                  OC8 = 0x1da
                    0x01da                  _OC8 = 0x1da
                    0x0240                  SPI1 = 0x240
                    0x0240                  _SPI1 = 0x240
                    0x0260                  SPI2 = 0x260
                    0x0260                  _SPI2 = 0x260
                    0x0220                  UART1 = 0x220
                    0x0220                  _UART1 = 0x220
                    0x0230                  UART2 = 0x230
                    0x0230                  _UART2 = 0x230
                    0x0001                  __MPLAB_BUILD = 0x1
START GROUP
LOAD c:/program files/microchip/mplab c30/bin/bin/../../lib\libpic30-coff.a
LOAD c:/program files/microchip/mplab c30/bin/bin/../../lib\libm-coff.a
LOAD c:/program files/microchip/mplab c30/bin/bin/../../lib\libc-coff.a
END GROUP
OUTPUT(ov9650Demo PIC24.cof coff-pic30)
LOAD jump_table
LOAD data_init
LOAD default_isr

_018e47e04a88ec30
                    0x0800        0x200
 _018e47e04a88ec30
                    0x0800        0x200 Objects - Image Decoders Demo\FSIO.o
                    0x0800                  gFATBuffer

_018e46904a88ec30
                    0x0a00        0x200
 _018e46904a88ec30
                    0x0a00        0x200 Objects - Image Decoders Demo\FSIO.o
                    0x0a00                  gDataBuffer

.nbss               0x0c00        0x1d6
 .nbss              0x0c00        0x194 Objects - Image Decoders Demo\FSIO.o
                    0x0c00                  defaultArray
                    0x0c0a                  defaultString
                    0x0c18                  gDiskData
                    0x0c36                  cwd
                    0x0c6c                  gFileTemp
                    0x0ca2                  tempCWDobj
                    0x0cd8                  dirCleared
                    0x0cda                  TempClusterCalc
                    0x0cde                  FSerrno
                    0x0ce0                  FatRootDirClusterValue
                    0x0ce4                  gTimeWrtDate
                    0x0ce6                  gTimeWrtTime
                    0x0ce8                  gTimeAccDate
                    0x0cea                  gTimeCrtDate
                    0x0cec                  gTimeCrtTime
                    0x0cee                  gTimeCrtMS
                    0x0cef                  gFileSlotOpen
                    0x0cf2                  gFileArray
 .nbss              0x0d94         0x42 Objects - Image Decoders Demo\Primitive.o
                    0x0dc4                  _fontHeight
                    0x0dc6                  _fontLastChar
                    0x0dc8                  _fontFirstChar
                    0x0dca                  _font
                    0x0dcc                  _fontOrientation
                    0x0dce                  _cursorY
                    0x0dd0                  _cursorX
                    0x0dd2                  _lineThickness
                    0x0dd4                  _lineType

.ndata              0x0dd6         0x2a
 .ndata             0x0dd6         0x2a Objects - Image Decoders Demo\Application.o
                    0x0dd6                  Couleur

.nbss               0x0e00         0x24
 .nbss              0x0e00         0x12 Objects - Image Decoders Demo\ImageDecoder.o
                    0x0e00                  IMG_pLoopCallbackFn
                    0x0e02                  IMG_blAbortImageDecoding
                    0x0e03                  IMG_bAlignCenter
                    0x0e04                  IMG_bDownScalingFactor
                    0x0e06                  IMG_wImageHeight
                    0x0e08                  IMG_wImageWidth
                    0x0e0a                  IMG_wHeight
                    0x0e0c                  IMG_wWidth
                    0x0e0e                  IMG_wStartY
                    0x0e10                  IMG_wStartX
 .nbss              0x0e12         0x12 Objects - Image Decoders Demo\DisplayDriver.o
                    0x0e12                  _line_mem_pitch
                    0x0e16                  _visualPage
                    0x0e17                  _activePage
                    0x0e18                  _clipBottom
                    0x0e1a                  _clipRight
                    0x0e1c                  _clipTop
                    0x0e1e                  _clipLeft
                    0x0e20                  _clipRgn
                    0x0e22                  _color

.ndata              0x0e24         0x12
 .ndata             0x0e24         0x12 Objects - Image Decoders Demo\FSIO.o
                    0x0e24                  cwdptr
                    0x0e26                  recache
                    0x0e27                  gBufferZeroed
                    0x0e28                  nextClusterIsLast
                    0x0e29                  gNeedDataWrite
                    0x0e2a                  gLastDataSectorRead
                    0x0e2e                  gBufferOwner
                    0x0e30                  gNeedFATWrite
                    0x0e32                  gLastFATSectorRead

.nbss               0x0e36          0x6
 .nbss              0x0e36          0x4 Objects - Image Decoders Demo\SD-SPI.o
                    0x0e36                  MDD_SDSPI_finalLBA
 .nbss              0x0e3a          0x2 Objects - Image Decoders Demo\Application.o
                    0x0e3a                  Counter

.ndata              0x0e3c          0x4
 .ndata             0x0e3c          0x2 Objects - Image Decoders Demo\Primitive.o
 .ndata             0x0e3e          0x2 Objects - Image Decoders Demo\DisplayDriver.o
                    0x0e3e                  _gpioStatus

.bss                0x0e40         0x88
 .bss               0x0e40         0x88 c:/program files/microchip/mplab c30/bin/bin/../../lib\libc-coff.a(rand.o)

.data               0x0ec8          0xa
 .data              0x0ec8          0xa c:/program files/microchip/mplab c30/bin/bin/../../lib\libc-coff.a(rand.o)
                    0x0ec8                  _Tls_setup__Randseed
                    0x0eca                  _Randseed
                    0x0ece                  _Tls_setup__Randinit
                    0x0ed0                  _Randinit

.const              0x86a8       0x23b2 load address 0x0006a8  
 .const             0x86a8       0x1584 Objects - Image Decoders Demo\GOLFontDefault.o
                    0x86a8                  L1191258975
                    0x9c28                  GOLFontDefault
 .const             0x9c2c        0xd6c Objects - Image Decoders Demo\Application.o
                    0x9c2c                  face
                    0x9c74                  pz
                    0x9c84                  py
                    0x9c94                  px
                    0x9ca4                  co
                    0xa244                  si
 .const             0xa998         0x66 Objects - Image Decoders Demo\SD-SPI.o
                    0xa998                  sdmmc_cmdtable
 .const             0xa9fe         0x4c Objects - Image Decoders Demo\JpegDecoder.o
 .const             0xaa4a         0x10 Objects - Image Decoders Demo\FSIO.o

.text             0x002a5a       0x7f46
 .text            0x002a5a       0x32c4 Objects - Image Decoders Demo\FSIO.o
                  0x002a5a                  Cluster2Sector
                  0x002aae                  ReadByte
                  0x002ab4                  LoadMBR
                  0x002bd2                  ReadWord
                  0x002bde                  ReadDWord
                  0x002c02                  LoadBootSector
                  0x002d4a                  DISKmount
                  0x002d82                  FSInit
                  0x002dfa                  GetFullClusterNumber
                  0x002e0e                  flushData
                  0x002e3a                  FSCreateMBR
                  0x002f8e                  FSformat
                  0x00347e                  Write_File_Entry
                  0x0034d2                  WriteFAT
                  0x0036b6                  ReadFAT
                  0x003882                  Cache_File_Entry
                  0x0039d8                  FILEget_next_cluster
                  0x003aa2                  FAT_erase_cluster_chain
                  0x003b5c                  LoadDirAttrib
                  0x003ba2                  CacheTime
                  0x003c36                  PopulateEntries
                  0x003cdc                  FATfindEmptyCluster
                  0x003d96                  EraseCluster
                  0x003df8                  FILECreateHeadCluster
                  0x003e5e                  CreateFirstCluster
                  0x003e9c                  FILEallocate_new_cluster
                  0x003f0c                  FindEmptyEntries
                  0x003f84                  CreateFileEntry
                  0x003fd4                  FSfclose
                  0x004070                  Fill_File_Object
                  0x00412a                  FILEopen
                  0x0041e8                  FILEfind
                  0x00431c                  FILEerase
                  0x004396                  FileObjectCopy
                  0x0043a4                  FSfseek
                  0x0044f0                  FSftell
                  0x0044f8                  FSrewind
                  0x00451c                  FSerror
                  0x004522                  FSattrib
                  0x00458a                  FSfwrite
                  0x004758                  FSfeof
                  0x004770                  FSfread
                  0x0048ca                  ValidateChars
                  0x004978                  FormatFileName
                  0x004a14                  FSremove
                  0x004aa2                  FSfopen
                  0x004c80                  FSrename
                  0x004d76                  FormatDirName
                  0x004e12                  chdirhelper
                  0x005046                  FSchdir
                  0x00504e                  GetPreviousEntry
                  0x005138                  FSgetcwd
                  0x00538a                  writeDotEntries
                  0x00543a                  CreateDIR
                  0x005500                  mkdirhelper
                  0x00571a                  FSmkdir
                  0x005722                  eraseDir
                  0x00578a                  rmdirhelper
                  0x005a9e                  FSrmdir
                  0x005aa8                  FindFirst
                  0x005bfc                  FindNext
 .text            0x005d1e       0x1136 Objects - Image Decoders Demo\JpegDecoder.o
                  0x005ed8                  JPEG_bDecode
 .text            0x006e54        0xea4 Objects - Image Decoders Demo\BmpDecoder.o
                  0x006e54                  BDEC_vResetData
                  0x006e76                  BDEC_bReadHeader
                  0x007034                  BMP_bDecode
 .text            0x007cf8        0xbd6 Objects - Image Decoders Demo\DisplayDriver.o
                  0x007cf8                  DelayMs
                  0x007d0e                  SetAddress
                  0x007d54                  SetRegB
                  0x007dac                  GetReg
                  0x007e2c                  GetRegW
                  0x007e44                  SetRegW
                  0x007e58                  SetRegL
                  0x007e76                  GetRegL
                  0x007e96                  GPIO_SPENA
                  0x007ea8                  GPIO_SPCLK
                  0x007eba                  GPIO_SPDAT
                  0x007ecc                  GPIO_SPRESET
                  0x007ede                  PutPixel
                  0x007f58                  GetPixel
                  0x007fca                  Bar
                  0x00806c                  ClearDevice
                  0x0080aa                  PutImage1BPP
                  0x0081d0                  PutImage4BPP
                  0x0082ec                  PutImage8BPP
                  0x0083fc                  PutImage16BPP
                  0x0084de                  PutImage
                  0x008548                  SPI_Write
                  0x008570                  SPI_SetReg
                  0x0085a2                  ResetDevice
                  0x00878a                  ssd1928_FloatWndInit
                  0x00880a                  ssd1928_FloatWndEnable
                  0x008826                  ssd1928_MainWndInit
                  0x008884                  ssd1928_FocusWnd
                  0x0088b2                  ssd1928_MainWndEnable
 .text            0x0088ce        0x972 Objects - Image Decoders Demo\Primitive.o
                  0x0088ce                  InitGraph
                  0x0088f8                  Arc
                  0x008c4e                  Line
                  0x008daa                  Bevel
                  0x008f6c                  FillBevel
                  0x009058                  DrawPoly
                  0x00908c                  SetFont
                  0x0090a4                  OutChar
                  0x009180                  OutText
                  0x0091a0                  OutTextXY
                  0x0091ba                  GetTextWidth
                  0x0091f0                  GetTextHeight
                  0x009200                  GetImageWidth
                  0x009220                  GetImageHeight
 .text            0x009240        0x7a4 Objects - Image Decoders Demo\Application.o
                  0x009240                  PixelOutput
                  0x009288                  Obj3D
                  0x00945c                  main
 .text            0x0099e4        0x70c Objects - Image Decoders Demo\jidctint.o
                  0x0099e4                  jpeg_idct_islow
 .text            0x00a0f0        0x44e Objects - Image Decoders Demo\ov9650.o
                  0x00a0f0                  camVideoPreview
                  0x00a16c                  camVideoStill
                  0x00a188                  camCmdWr
                  0x00a1b2                  camRegRd
                  0x00a1ea                  camHwInit
                  0x00a4e2                  camInit
 .text            0x00a53e        0x310 Objects - Image Decoders Demo\SD-SPI.o
                  0x00a53e                  MDD_SDSPI_MediaDetect
                  0x00a546                  MDD_SDSPI_ReadSectorSize
                  0x00a548                  MDD_SDSPI_ReadCapacity
                  0x00a54e                  MDD_SDSPI_InitIO
                  0x00a558                  CloseSPIM
                  0x00a55c                  MDD_SDSPI_ShutdownMedia
                  0x00a562                  WriteSPIM
                  0x00a570                  MDD_SDSPI_ReadMedia
                  0x00a580                  SendMMCCmd
                  0x00a650                  MDD_SDSPI_SectorRead
                  0x00a6e2                  MDD_SDSPI_SectorWrite
                  0x00a768                  MDD_SDSPI_WriteProtectState
                  0x00a770                  Delayms
                  0x00a790                  OpenSPIM
                  0x00a7a6                  MDD_SDSPI_MediaInitialize
 .text            0x00a84e         0xc8 Objects - Image Decoders Demo\ImageDecoder.o
                  0x00a84e                  ImageDecoderInit
                  0x00a862                  ImageLoopCallbackRegister
                  0x00a866                  ImageDecode
                  0x00a8a2                  IMG_vSetboundaries
 .text            0x00a916         0x8a Objects - Image Decoders Demo\SSD1928_I2C.o
                  0x00a916                  ssd1928_I2C_Init
                  0x00a92e                  ssd1928_I2C_Wait
                  0x00a952                  ssd1928_I2C_Ctl
                  0x00a966                  ssd1928_I2C_Write
                  0x00a96c                  ssd1928_I2C_Read

.dinit            0x00a9a0         0x8a
 .dinit           0x00a9a0         0x8a data_init

.isr              0x00aa2a          0x2
 .isr             0x00aa2a          0x2 default_isr
                  0x00aa2a                  _DefaultInterrupt
